:0200000480007A
:10000000B72F0000938F0F8073900F3015A8130047
:100010000000130000001300000013000000130094
:100020000000130000001300000013000000130084
:100030000000130000001300000013000000010086
:10004000970200009382020C73905230814001416C
:100050008141014281420143814301448144014580
:100060008145014681460147814701488148014950
:100070008149014A814A014B814B014C814C014D20
:10008000814D014E814E014F814F971102009381A6
:10009000E1D8170502001305E56697A503009385CF
:1000A00025860146112217050200130525509705E4
:1000B0000200938565560146C52817B50300130550
:1000C000658497C503009385A58337B6ABAB13064C
:1000D000B6BAD92817C103001301C182EF80B02A34
:1000E000860293D21200F512638802008242110147
:1000F0006F00001073002030824211017300203025
:10010000711116C0F3222034E3CC02FC82421101AB
:10011000130141F806C20AC40EC612C816CA1ACC88
:100120001ECE22D026D22AD42ED632D836DA3ADCC7
:100130003EDEC2C0C6C2CAC4CEC6D2C8D6CADACC97
:10014000DECEE2D0E6D2EAD4EED6F2D8F6DAFADCA7
:10015000FEDE73252034F32510340A8601A07310C7
:10016000153492402241B2414242D2426243F243AC
:10017000025492542255B2554256D2566257F25703
:10018000064896482649B649464AD64A664BF64B33
:10019000065C965C265DB65D465ED65E665FF65F83
:1001A0001301C1077300203010C16374B50011053D
:1001B000E5BF828000000000000000000000000099
:1001C000000000000000000000000000000000002F
:1001D000000000000000000000000000000000001F
:1001E000000000000000000000000000000000000F
:1001F000197106C00AC20EC412C616C81ACA1ECC8D
:1002000022CE26D02AD22ED432D636D83ADA3EDCC6
:1002100042DEC6C0CAC2CEC4D2C6D6C8DACADECC96
:10022000E2CEE6D0EAD2EED4F2D6F6D8FADAFEDCA6
:100230009702020083A2C23A23A02200F3221034C4
:1002400096DEEF00002B1701020003216139024105
:10025000F65273901234B72200009382028873A082
:10026000023082403242C2425243E24372448254DC
:100270001255A2553256C2565257E2577258864806
:100280001649A649364AC64A564BE64B764C865C1A
:10029000165DA65D365EC65E565FE65F0961730059
:1002A0002030970202009382E24523A0120023A28D
:1002B000220023A4320023A6420023A8520023AA2E
:1002C000620023AC720023AE820023A0920223A21C
:1002D000A20223A4B20223A6C20223A8D20223AA06
:1002E000E20223ACF20223AE020323A0120523A2F2
:1002F000220523A4320523A6420523A8520523AADA
:10030000620523AC720523AE820523A0920723A2C7
:10031000A20723A4B20723A6C20723A8D20723AAB1
:10032000E20723ACF207EF4050301701020003212F
:10033000212B0241F65273901234B72200009382AF
:10034000028873A0023082403242C2425243E243EA
:10035000724482541255A2553256C2565257E25731
:10036000725886481649A649364AC64A564BE64B45
:10037000764C865C165DA65D365EC65E565FE65FB1
:10038000096173002030970202009382A23783A094
:10039000020003A1420083A1820003A2C20083A243
:1003A000020103A3420183A3820103A4C20183A427
:1003B000020203A5420283A5820203A6C20283A60B
:1003C000020303A7420383A7820303A8C20383A8EF
:1003D000020403A9420483A9820403AAC20483AAD3
:1003E000020503AB420583AB820503ACC20583ACB7
:1003F000020603AD420683AD820603AEC20683AE9B
:10040000020703AFC20983AF820782807370043092
:10041000197106C00AC20EC412C616C81ACA1ECC6A
:1004200022CE26D02AD22ED432D636D83ADA3EDCA4
:1004300042DEC6C0CAC2CEC4D2C6D6C8DACADECC74
:10044000E2CEE6D0EAD2EED4F2D6F6D8FADAFEDC84
:100450009702020083A2C21823A0220086DEEF20AA
:100460004037170102000321A1170241F652739091
:100470001234B72200009382028873A002308240B7
:100480003242C2425243E243724482541255A25550
:100490003256C2565257E257725886481649A649F4
:1004A000364AC64A564BE64B764C865C165DA65DD0
:1004B000365EC65E565FE65F09617300203073707A
:1004C000043001A07310453082807325403073F0F2
:1004D00043308280970700009387A7FE232EB5FE46
:1004E0002322C5FA232635F82320F5F8130505F84D
:1004F0008280411106C6EF407010EF10301501E503
:10050000B24041018280B24041016F20802C9307AC
:1005100085007D575CC118C55CC51CC9232005003A
:1005200082802328050082805C41DCC1984798C501
:1005300098474CC38CC788C91C4185071CC1828061
:100540009041FD57130785006314F60039A83E87D4
:100550005C439443E37DD6FEDCC18CC798C54CC395
:1005600088C91C4185071CC1828018495C43EDB7CE
:10057000584114451C4914C71845544154C3D84325
:100580006314A7001845D8C32328050088437D15A8
:1005900088C382803041AE8701CE4C455841B29528
:1005A0004CC563E4E5000C414CC53E856F30902995
:1005B0008280411122C406C62A8426C2EF20101B65
:1005C0003C44635BF0025C5085CB9304440209A871
:1005D0003C44FD173CC43C446350F0025C5089CF5E
:1005E0002685EF2020616DD5EF2010013C44FD17DA
:1005F0003CC43C44E344F0FEFD573CC4EF2050199A
:10060000EF20D0167C40635BF0021C4885CB93043E
:10061000040109A87C40FD177CC07C406350F002B7
:100620001C4889CF2685EF20E05C6DD5EF20C07C8B
:100630007C40FD177CC07C40E344F0FEFD577CC04D
:100640002244B240924441016F20901429CD0111FF
:1006500022CC2A8406CE26CA4AC84EC62E89EF204E
:10066000F01024404C5C832904002685EF808036FE
:100670007D57232C0402B3079540CE974E9578C042
:1006800048C0232434015CC438C4631109021C48E7
:100690008DE7EF20F00FF2406244D2444249B24964
:1006A0000545056182807370043001A013050401C3
:1006B000B93D13054402A13DE9BF13050401EF2034
:1006C00060538547E317F5FC9133E1B701E573709B
:1006D000043001A0011126CA4AC84EC606CE22CC5B
:1006E000AA842E89B289A5C9EF80C02E13055505AD
:1006F000EF30007D2A8435C5930745051CC144DCD5
:1007000023202405EF20900624404C5C032904009C
:100710002685EF80202CFD56232C0402B30795403C
:100720003307A900CA9774C058C05CC434C4130509
:10073000040123242401E13B13054402C93BEF20BB
:100740003005230834052285F2406244D2444249F0
:10075000B2490561828013054005EF3060762A8436
:1007600001E57370043001A000C051BF01E5737052
:10077000043001A06375B5007370043001A041110D
:1007800022C409462E84814506C6893711C500DD7D
:10079000B2402244410182807370043001A05D7137
:1007A00086C6A2C4A6C2CAC04EDE52DC56DA5AD8E9
:1007B0005ED632C6630A051C6382051C89476399AD
:1007C000F600585D85476305F7007370043001A09B
:1007D0003689AE842A84EF20A06411E5B24781C730
:1007E0007370043001A0EF206078185C5C5C014BF2
:1007F000894BFD59130A0401930A44026365F70CFF
:1008000063077919B2476381072463150B00280831
:10081000EF206051EF20C077EF10005AEF200075F5
:100820007C4063943701232204043C4463943701E1
:1008300023240404EF20C0756C002808EF20C0506A
:10084000631E051EEF208072185C5C5C630CF70A67
:10085000EF200074EF2080713C44634FF00039A812
:100860005685EF20203919C1EF2000593C44FD176F
:100870003CC43C446354F0005C50FDF32324340535
:10088000EF200071EF20806E7C40634FF00039A8AC
:100890005285EF20203619C1EF2000567C40FD170D
:1008A0007CC07C406354F0001C48FDF323223405D7
:1008B000EF20006EEF104075054BEF20206B185CA9
:1008C0005C5CE37FF7F230406305060C631F09129E
:1008D0000844A685EF3000771C4434405840B69752
:1008E0001CC463EAE70A1C5C14405850850714C412
:1008F0001CDC5DC713054402EF20C02F8547631140
:10090000F50AC9A8EF20C068B2455285EF20401013
:10091000EF20C0653C44634FF00039A85685EF20B6
:10092000602D19C1EF20404D3C44FD173CC43C44B0
:100930006354F0005C50FDF323243405EF20406540
:10094000EF20C0627C40634FF00039A85285EF2051
:10095000602A19C1EF20404A7C40FD177CC07C40D2
:100960006354F0001C48FDF323223405EF2040625D
:10097000EF10806931F1593C054B81B73C41E38F61
:1009800007E27370043001A07370043001A030409E
:1009900021E61C4085C71C5C585085071CDC39FBD0
:1009A000EF20005F0545B640264496440649F259BB
:1009B000625AD25A425BB25B616182804840EF204A
:1009C00040521C5C58502322040085071CDCE313B2
:1009D00007F279D5253CE9B74844A685EF30806613
:1009E0003C4058441440B307F0403E9758C4637CE1
:1009F000D7025840BA975CC409475C506306E902C5
:100A0000185C050718DCC9DFF5B54844A685EF304A
:100A100060633C4058441440B307F0403E9758C4CC
:100A2000E37CD7FCF9B75C50185C79DB185C7D1768
:100A300018DC185C050718DCA5D76DBD2285953E2E
:100A4000EF10805C014585B7EF2080540145A1BFC0
:100A5000411126C2AA841305400522C406C6EF3000
:100A600020462A8415CD232C0502FD577CC105475D
:100A7000410558DC3CC42322040023200400232425
:100A80000400232604002320040423089404413492
:100A900013054402AD3C8146014681452285013360
:100AA0002285B24022449244410182800DC5411109
:100AB00022C426C206C64AC0032945002A84EF2064
:100AC00060358144630CA900B24022442685024966
:100AD0009244410182807370043001A05C448544DB
:100AE000FD175CC4F5F381460146814522854539F1
:100AF000E1BF31CDA1C9011122CC26CA4AC852C4D6
:100B000006CE4EC68947B68432892E8A2A846399D6
:100B1000F600585D8547630FF7047370043001A039
:100B20006D32185C5C5CAA896366F70281444E856D
:100B3000513AF240624426854249D244B249224A9F
:100B4000056182803C41C5DB7370043001A0737085
:100B5000043001A0304041E21C40D5CB1C5C7D57E5
:100B600085071CDC3C446387E7083C4485448507D3
:100B70003CC475BF993A185C5C5CAA89636DF70246
:100B8000304079DA4844D285EF30C04B3C4058447D
:100B90001440B307F0403E9758C46375D7005840DF
:100BA000BA975CC48947E39BF4FA1C5CC5DB1C5C08
:100BB000FD171CDC65B7304045D24844D285EF3084
:100BC00060483C4058441440B307F0403E9758C436
:100BD000E367D7FCD9BFDDF40844D285EF30804607
:100BE0001C4434405840B6971CC4E3E9E7F61C4067
:100BF0001CC4ADB75C5085449DDB13054402EF1067
:100C0000707F15D5E30509F2232099000DB7484000
:100C1000EF20202D2322040091B721CD3C4181C734
:100C20007370043001A01C41A1CB011122CC26CA53
:100C30002A844AC84EC606CE2E894138185C5C5CB0
:100C4000AA898144637DF7001C5C7D5785071CDC05
:100C50003C446388E7023C44854485073CC44E8598
:100C60009530F240624426854249D244B24905613A
:100C700082807370043001A05C41C5DB7370043066
:100C800001A05C5099E38544D9BF13054402EF10DD
:100C9000707675D9E30909FE85472320F900E5B789
:100CA000397106DE22DC26DA4AD84ED652D456D224
:100CB00032C66302051C638A051AB68AAE892A8485
:100CC000EF20001611E5B24781C77370043001A010
:100CD000EF20C0291C5C63920714B247638E070A99
:100CE0002808EF204004FD5413094402130A0401AC
:100CF000EF20002AEF10400CEF2040277C40639447
:100D00009700232204043C446394970023240404A2
:100D1000EF2000286C002808EF200003631305185B
:100D2000EF20C0241C5CADCFEF208026EF200024F4
:100D30003C44634FF00039A84A85EF10B06B19C1ED
:100D4000EF20800B3C44FD173CC43C446354F0004E
:100D50005C50FDF324C4EF20A023EF2020217C4031
:100D6000634FF00039A85285EF10D06819C1EF2009
:100D7000A0087C40FD177CC07C406354F0001C48F8
:100D8000FDF364C0EF20C020EF100028EF20001E0C
:100D90001C5CC1E7B247A9FFEF20801F014555A0A9
:100DA000EF20001F1C40DDC7B2454A85EF105046BA
:100DB000EF20C01B3C44634FF00039A84A85EF1078
:100DC000706319C1EF2040033C44FD173CC43C4410
:100DD0006354F0005C50FDF324C4EF20601BEF204F
:100DE000E0187C40634FF00039A85285EF10906006
:100DF00019C1EF2060007C40FD177CC07C4063542B
:100E0000F0001C48FDF364C0EF208018EF10C01FF5
:100E100031C9EF20A0151C5CB5DFCE852285444486
:100E2000EFF04FF7639C0A041C5C1840FD171CDCB4
:100E300001E7EF20601A48C01C48A1EFEF204015E1
:100E40000545F2506254D2544259B259225A925A2C
:100E500021618280EF2080114840EF10707EEF20EA
:100E6000201399B7EFF08FDA6DB73C41E38707E4C1
:100E70007370043001A07370043001A05C5044C44E
:100E8000D5DF13054402EF10F0564DD9EFF00FD81F
:100E900075B713050401EF10F0558547E310F5FA17
:100EA000F5B72285EFF0EFF0EF100016014551BFC6
:100EB0001DC9411122C44AC006C626C244412E891A
:100EC0002A84EF1030756383A40281464A868145E7
:100ED0002285F93385476300F502B24022449244EB
:100EE0000249410182807370043001A05C440545D1
:100EF00085075CC4DDB75C4485075CC4F9BF15CDCC
:100F0000ADC9011122CC26CA4AC84EC652C42A8491
:100F100006CE3289AE89EFF04FDB1C5C2A8A814411
:100F200085E35285EFF00FDAF240624426854249AC
:100F3000D244B249224A056182807370043001A014
:100F4000304001CE4C445C40B2954CC463E4F500A3
:100F50000C404CC44E85EF30E00E1C5C7D57FD17F5
:100F60001CDC7C40638CE7007C40854485077CC0AA
:100F70004DBF3C41D9D77370043001A01C4899E3A0
:100F8000854445B713050401EF10D04675D9E30930
:100F900009FE85472320F900E5B721C93C41A1CDD1
:100FA000A1CB011122CC26CA4AC852C42A8406CE3B
:100FB0004EC62E8AEFF06FD11C5C2A89814491CBFA
:100FC0008329C400D2852285EFF0CFDC8544232617
:100FD00034014A85EFF00FCFF24062442685424942
:100FE000D244B249224A056182807370043001A064
:100FF0007370043001A0EDDF7370043001A001E5CF
:101000007370043001A0411122C42A8406C6EF1077
:10101000F075005CEF10D077B24022852244410188
:10102000828001E57370043001A0411106C622C41C
:101030002A84EF10B0731C5C405C1D8CEF1050755F
:101040002285B24022444101828019C1085D82801C
:101050007370043001A01DCD979703009387878696
:10106000D843630CE502D847630CE504D84B63070B
:10107000E504D84F6302E504D853630DE502D85761
:101080006308E502D85B6303E502D85F630EE50001
:101090006F2030757370043001A001470E07BA97B6
:1010A00023A007006F20F0731D47CDBF1947FDB780
:1010B0001547EDB71147DDB70D47CDB70947F9BF64
:1010C0000547E9BF684582806CC5828003450505F8
:1010D000828009C5085D1335150082807370043065
:1010E00001A019C51C5D485D1D8D1335150082805A
:1010F0007370043001A0978703009387A77C9843FF
:1011000005C3984705C7984B05C7984F05C798531F
:1011100005C7985705C7985B15C7985F15C38280A8
:1011200001470E07BA978CC3C8C382800547D5BF55
:101130000947C5BF0D47F5B71147E5B71547D5B7FF
:101140001D47C5B71947F1BF978703009387877776
:10115000D8436308E502D847630BE502D84B630A1E
:10116000E502D84F6309E502D8536308E502D85772
:101170006307E502D85B6308E502D85F6303A70253
:10118000828001470E07BA9723A007008280054797
:10119000D5BF0947C5BF0D47F5B71147E5B7154797
:1011A000D5B71D47C5B71947F1BF411122C426C2A3
:1011B0004AC02A8406C6AE843289EF10305B78407C
:1011C000FD576314F700232204043844FD576314C9
:1011D000F70023240404EF10B05B1C5C99E74A86F7
:1011E000A68513054402EF10B015EF1030583C44AB
:1011F000635BF0025C5085CB9304440209A83C4435
:10120000FD173CC43C446350F0025C5089CF2685F6
:10121000EF10501E6DD5EF10303E3C44FD173CC41E
:101220003C44E344F0FEFD573CC4EF107056EF1011
:10123000F0537C40635BF0021C4885CB93040401AF
:1012400009A87C40FD177CC07C406350F0021C481C
:1012500089CF2685EF10101A6DD5EF10F0397C403C
:10126000FD177CC07C40E344F0FEFD577CC0224467
:10127000B2409244024941016F10905197F701002A
:1012800093870736944317F7010013072734184351
:10129000C8C2636EE502411122C406C617F70100F9
:1012A0001307C7332A8408438C439105EFF04FA9F5
:1012B00097F701009387C72F9C436376F40097F755
:1012C000010023A7872EB24022444101828017F7F4
:1012D00001001307673008438C4391056FF04FA658
:1012E00097F701009387C72F984394437C43FD17DA
:1012F0007CC3FC4299E37360043082801DC1797124
:101300004ECE56CA06D6BE8A22D426D24AD052CC57
:101310005AC85EC69147BA8963F8E7007370043013
:1013200001A07370043001A02A8BAE843289B68B81
:10133000428A6308082213050006EF2070382A84C9
:10134000630C05200A09232845034A869305500AA1
:101350005285EF20305D03C704001C587119230A21
:10136000E40203C704003E991379C9FF79C783C714
:101370001400A30AF40283C71400E1C383C7240046
:10138000230BF40283C72400CDCB83C73400A30B07
:10139000F40283C73400D5C383C74400230CF4028E
:1013A00083C74400D9CB83C75400A30CF40283C77E
:1013B0005400C1C783C76400230DF40283C76400CF
:1013C000ADCF83C77400A30DF40283C77400B5C703
:1013D00083C78400230EF40283C78400B9CF83C778
:1013E0009400A30EF40283C79400A1CB83C7A4008A
:1013F000230FF40283C7A400A9C383C7B400A30FBB
:10140000F40283C7B40095CB83C7C4002300F4045F
:1014100083C7C4009DC383C7D400A300F40483C75B
:10142000D40081CF83C7E4002301F40483C7E40020
:1014300089C783C7F400A301F404130A440052854A
:10144000A30104042326340323283405232A040497
:10145000EFF02F8D13058401EFF0AF8C9547B38724
:101460003741232C040400C81CCC40D023220404A0
:10147000232E04045E86DA854A85EFF0AF8508C026
:1014800063840A0023A08A007370043017F90100F6
:10149000130949138327090097F401009384441426
:1014A00091C798409C407C4385077CC317F7010097
:1014B000130707121C43850797F6010023AAF610AD
:1014C0009C40CDCB8327090089EB9C40DC5763E629
:1014D000F90097F7010023A5871097F7010093877C
:1014E000670D9C4317F701001307070E4854184374
:1014F000850797F6010023AFF60A3CC46376A70080
:1015000097F7010023A2A70CD145EF70A04C97F7E5
:1015100001009387E7263E95D285EFF0EF80832781
:10152000090089C79C40FC436395070E8327090087
:10153000054499C79C40DC5763F43701EFE01FED89
:101540002285B250225492540259F249624AD24A38
:10155000424BB24B456182805285EF2090287D54EA
:10156000C5B713152600EF20B0152A8AE31505DC50
:101570007D54F9B797F7010023A4870618438547E0
:10158000E31DF7F417F501001305851FEFE03FF8A1
:1015900017F5010013050520EFE07FF717F50100AF
:1015A00013058520EFE0BFF617F5010013050521AF
:1015B000EFE0FFF517F5010013058521EFE03FF59A
:1015C00017FB0100130B0B225A85EFE05FF497FA2B
:1015D0000100938A6A225685EFE07FF317F5010038
:1015E0001305C522EFE0BFF217F5010013054523EF
:1015F000EFE0FFF117F501001305C523EFE03FF120
:1016000097F7010023AC67FD97F7010023A657FD6C
:10161000E9B5984094407C43FD177CC3FC42E397B6
:1016200007F07360043019B7411122C406C626C200
:101630004AC02A847370043097F40100938484F8BC
:101640009C40F9E311E497F70100938767F9804321
:10165000130944004A85EFE0BFF11C5489C7130504
:101660008401EFE0FFF0CA8517F501001305451B63
:10167000EFE09FEB97F701009387C7F5984397F743
:101680000100938727F39C43050797F6010023A3E6
:10169000E6F49840850797F6010023ADF6F001CBFC
:1016A00097F701009387C7F39843784349EF9C402D
:1016B000B1C797F701009387A7F29843630F870894
:1016C00073700430984039EB17F70100130707F1E6
:1016D00014439442A5E27D5797F6010023AAE6EC55
:1016E000984009CF9843784311CB984394437C4367
:1016F000FD177CC3FC4299E373600430B24022447E
:10170000924402494101828097F70100938747ED97
:1017100098439C437C4385077CC32DB794439843EF
:10172000F8420507F8C217F70100130727EB144327
:101730009442D5D2184358475847584397F601006A
:1017400023A8E6E671BF984394437C43FD177CC30E
:10175000FC42B1FF7360043099BF97F70100938793
:10176000E7E49C4381C77370043001A02244B24077
:101770009244024941016FE07FC941C517F701005A
:10178000130707E614438147638BA606411106C67B
:1017900022C426C27370043097F60100938686E255
:1017A0009C4291C710431C437C4285077CC29C42EB
:1017B000AA84404981C71C43FC43B9E797F701005D
:1017C0009387C7E19C43638A870497F70100938757
:1017D000A7E09C436383870497F7010093878705FD
:1017E0006308F40297F70100938787036300F4020C
:1017F0008547B240224492443E85410182803E8525
:1018000082807370043001A0E13C4DBF9147D5B791
:101810009C5493B717008907E9BF8947D9BF7370F4
:10182000043097F701009387E7D9984309EF15C56E
:101830009C43485581CB97F70100938767DA98431B
:10184000784315E3828017F70100130767D9144323
:101850001843F8420507F8C261FD17F701001307A6
:1018600027D80843F1B7984394437C43FD177CC3C2
:10187000FC42E9FB736004308280411122C42A8457
:1018800006C6EFE09FC411E497F70100938747D5A0
:1018900080434054EFE01FC3B240228522444101FF
:1018A0008280914763F5B7007370043001A0011185
:1018B00022CC06CE26CA4AC84EC652C42A847370A9
:1018C000043017F901001309E9CF83270900CDEF90
:1018D00071C43C486388F50817F70100130747D027
:1018E00063FCB7001443638B860C18434457B3B4AE
:1018F000950093C4140029A00443818C93B4140070
:1019000058546383E70A1C4C2CC863C607009547EC
:10191000B385B7400CCC93172700BA97584897F96E
:1019200001009389E9E58A07CE97631AF702130A43
:1019300044005285EFE0DFC397F701009387C7C8E3
:1019400048549C4363F6A70097F7010023AEA7C64F
:10195000D145EF702008D2854E95EFE0FFBC99C0CD
:10196000EFE0DFAA8327090081CB97F70100938777
:1019700027C79C43FC439DEBF2406244D24442495A
:10198000B249224A0561828097F70100938747C5D3
:1019900098439C437C4385077CC305FC97F7010073
:1019A000938707C4804335B74CD4B1BF6244F2403B
:1019B000D2444249B249224A05611DB2814489B7E5
:1019C00025C1011126CA97F40100938464C19C408B
:1019D00006CE22CC4AC84EC6638DA702737004306F
:1019E00017F90100130909BE8327090091C7984020
:1019F0009C407C4385077CC3584997F70100938737
:101A000067E36302F7028327090081C79C40FC4318
:101A1000A5EBF2406244D2444249B249056182805A
:101A20007370043001A01C5517F70100130707DE7F
:101A3000E38BE7FCE9FB930945002A844E85EFE040
:101A40003FB397F70100938727B848549C4363F648
:101A5000A70097F7010023A9A7B6D145EF609077BB
:101A600097F701009387C7D13E95CE85EFE0DFABB6
:101A70009C405854DC57E368F7F8EFE03F9961B7B2
:101A80006244F240D2444249B249056191B815CD51
:101A9000011122CC26CA4EC62A8406CE4AC8EFE0DF
:101AA000DFA2584897F701009387C7D8AA898144D5
:101AB0006300F7024E85EFE0FFA0F2406244268506
:101AC0004249D244B249056182807370043001A05A
:101AD0001C5417F50100130565D3E38DA7FCF9FB32
:101AE00097F70100938787AC9C43A9EB97F7010018
:101AF000938707AF9C43445413094400DC574A853D
:101B0000B3B4F400EFE0DFA697F701009387C7AB0B
:101B100048549C4393C4140063F6A70097F7010050
:101B200023A4A7AAD145EF60F06A97F70100938735
:101B300027C5CA853E95EFE03F9FADBF9305840161
:101B4000EFE09F9E85BF0111056506CE22CC26CA17
:101B50004AC84EC652C456C2EF208036630E051CDA
:101B6000AA8413050006EF20A0352A84630A051E07
:101B700005669305500A04D92685EF20A05A04581B
:101B80008567F117BE94B7474C45938797449309EF
:101B900044005CD84E85230C0402A30104042326D0
:101BA000040223280404232A0404EFE09F9713056A
:101BB0008401EFE01F979547232C0404F19800C897
:101BC0001CCC40D023220404232E04040146971584
:101BD00000009385E5B12685EFE0DF8F08C07370C4
:101BE000043017F901001309E99D8327090097F4D0
:101BF00001009384E49E91C798409C407C438507F4
:101C00007CC317F701001307A79C1C43850797F6B1
:101C1000010023AFF69A9C40C9C38327090081EBDA
:101C20009C40DC5789E797F7010023AB879A97F729
:101C30000100938727989C4397F601009386C698E6
:101C400058549442850717F601002325F6963CC4A4
:101C500063F6E60097F7010023A8E796931727009D
:101C6000BA978A0717F50100130585B13E95CE8511
:101C7000EFE09F8B8327090081C79C40FC43F1E77D
:101C80008327090091C39C40EF10F0498547630406
:101C9000F50E5DE17370043001A097F7010023A1F8
:101CA000879418438547E314F7F817F501001305E7
:101CB00025ADEFE0DF8517F501001305A5ADEFE0D9
:101CC0001F8517F50100130525AEEFE05F8417F5BA
:101CD00001001305A5AEEFE09F8317F50100130582
:101CE00025AFEFE0DF8297FA0100938AAAAF56850D
:101CF000EFE0FF8117FA0100130A0AB05285EFE006
:101D00001F8117F50100130565B0EFE05F8017F53F
:101D100001001305E5B0EFE08FFF17F50100130593
:101D200065B1EFE0CFFE97F7010023A9578B97F736
:101D3000010023A3478BE5BDF2406244D2444249EF
:101D4000B249224A924A05618280984094407C437D
:101D5000FD177CC3FC42E39507F2736004300DB7B6
:101D60006244F2404249B249224A924A2685D2440C
:101D700005616F20002773700430FD5717F70100CD
:101D80002328F782624497F7010023ADA782F2402F
:101D9000D2444249B249224A924A97F7010023A706
:101DA000078205616FE0EFCF7370043097F7010091
:101DB00023AA07806FE02FDD17E701001307077FD5
:101DC0001C4385071CC382807370043097E70100B1
:101DD0009387477F984305E317E701001307077FC1
:101DE00008439C4381CB97E701009387677F984323
:101DF000784301EF828017E701001307677E1443E1
:101E00001843F8420507F8C2C1BF984394437C4386
:101E1000FD177CC3FC42F9FF7360043082804111DE
:101E200006C622C4EFE06FEA97E701009387077ABE
:101E30008043EFE02FE9B2402285224441018280B5
:101E400097E701009387C77888438280797106D627
:101E500022D426D24AD04ECE52CC56CA5AC85EC6DA
:101E600097E70100938787749C43B1EF17E7010060
:101E70001307C7751C43850797E6010023A8F6746E
:101E8000832A0700638F0A0697E70100938747724A
:101E90009C43814463F1FA0897F901009389498EC4
:101EA00017EA0100130ACA7383270A008546D85728
:101EB00093172700BA978A07BE9983A7090063FF83
:101EC000F600854421A897E701009387676F9C433C
:101ED0008144850717E701002324F76E97E7010087
:101EE0009387C76D9C4391C38544B2502254268585
:101EF00002599254F249624AD24A424BB24B45616E
:101F0000828017E401001304646D1C409C43DDC310
:101F10007370043001A017E401001304246C97F9D6
:101F200001009389E98517EA0100130A6A6B17EB30
:101F30000100130B6B691C409C43B5C31C40DC477C
:101F400003A9C70083274900930B49005E8563EE10
:101F5000FA04EFE0EFE1832789021305890199C3B1
:101F6000EFE00FE18327C90203270B00DE851395FD
:101F700027003E950A054E956376F70017E70100A6
:101F80002324F764EFE04FDA83270A000327C9020E
:101F9000DC57E362F7FA1C4085449C43C5F3FD57C8
:101FA00017E701002326F76001B717E70100232197
:101FB000F760DDBD17E70100130707621C401843F7
:101FC00097E6010023ACE66017E701002326F760DF
:101FD00097E701009387475E9C43850717E7010059
:101FE000232CF75C1C409C4399E7FD5717E7010041
:101FF0002320F75C51BD1C40DC47DC47DC4317E77E
:1020000001002327F75A49B597E701009387075A3C
:10201000984301E77370043001A0011106CE22CC71
:1020200026CA4AC84EC652C456C25AC0737004303B
:1020300097E4010093840459984061EB98437D171D
:1020400097E6010023A4E6569C43D9EB97E70100ED
:10205000938707589C43C9C797EA0100938A4A723D
:1020600017EA0100130A4A5617E9010013094957F4
:10207000854919A83385EA00EFE00FCB83270900D3
:102080005854DC576379F70483A7CA08C1CF83A7E4
:102090008A09C04713058401EFE08FCD130B44007C
:1020A0005A85EFE0EFCC5C5483260A00DA8513955D
:1020B00027003E950A052A875695E3FDF6FA17E7AD
:1020C00001002323F750EFE02FC68327090058545F
:1020D000DC57E36BF7FA97E7010023A1374F6DB7A1
:1020E00001449C4081CB97E701009387674F9C4355
:1020F000FC4395E72285F2406244D2444249B2490A
:10210000224A924A024B0561828017E701001307B9
:10211000274D14431843F8420507F8C205B7EFF0FE
:102120002F9CC9BF17E40100130484491C4095C3C8
:102130001C40054999CF193B09C597E7010023AF1A
:1021400027471C40FD1717E70100232BF7461C40CB
:10215000FDF397E701009387674698438547E311AE
:10216000F7F8EFE0AFAA0544ADBF11CD81E573707C
:10217000043001A017E70100130747431C4399C728
:102180007370043001A07370043001A0411122C4A7
:1021900006C614431841850617E601002328D640D9
:1021A00097E601009386864294423304B70000C14B
:1021B00063F7E602637FE40063FD860097E70100B2
:1021C0009387074288431105EFE08FBA2285EFF02D
:1021D000EF8A1D3D01C9B240224441018280E36F74
:1021E000E4FCD9BF2244B24041016FE02FA211C9E3
:1021F00017E701001307873B1C4391C77370043036
:1022000001A06FE0AFA0411106C622C41843AA87FF
:10221000050797E6010023ABE63897E601009386B1
:10222000263C17E701001307673A18438842330436
:10223000F7001105EFE0CFB32285EFF02F84E933EB
:1022400011E52244B24041016FE04F9CB24022446C
:1022500041018280411122C406C697E7010093879D
:10226000E7349C430144850717E701002320F73436
:1022700097E701009387C7359C4363E3F50C17EE9E
:102280000100130E6E5597E201009382A24E0144A5
:102290000147854F1303500A21A0311E6387C20DE9
:1022A00083278EFFBA85F5DB8327CEFFDC43232E01
:1022B000FEFE6382C71B03AFC700DC432A97814E33
:1022C000232EFEFE6385C70783A8C70093874803B4
:1022D000232017015CC383A788042326F7011CC7AA
:1022E00083A7C8021CCB83A70805232C07005CCB5F
:1022F00003A8080383470800639A6704C287850719
:1023000083C60700B3850741E38B66FE8981C2055A
:10231000C181231EB700850E1307070263001F0546
:102320008327CEFFDC43232EFEFEE39FC7F98327DE
:102330004E00232EFEFE49BF1A9419C22320060028
:10234000E1312285B2402244410182808145231E31
:10235000B700850E13070702E3141FFD76941317C9
:102360005400311EBA85E39DC2F397E701009387BD
:10237000E72603AE070083270E00FDE397E7010081
:102380009387872503AE070083270E0063980716FF
:1023900017EE0100130ECE3E83270E0A639D071E23
:1023A00083274E0BD9DB83278E0B97EE0100938E8C
:1023B000EE48DC4317E701002320F7486381D73359
:1023C00083AFC700DC433307B500014397E6010044
:1023D00023A4F6460D4F89429308500A6386D70717
:1023E000C8479307450308C35CC33C452326E70160
:1023F0001CC75C551CCB1C5599C3232657003C4970
:10240000232C07005CCB0328050383470800639552
:10241000172BC287850783C60700B3850741E38B67
:1024200016FF8981C205C181231EB700050313076A
:102430000702E383AFF083278E0BDC4397E60100AE
:1024400023ACF63EE39ED7F983270E0C97E60100F6
:1024500023A4F63E71B783274E00232EFEFEA1BDB6
:1024600083274E00130F8E00D4432322DE00638C9B
:10247000E625B307E500D84283A2C600814E232299
:10248000EE00894F1303500A6305EF068328C70047
:102490001387480323A01701D8C303A7880423A6E2
:1024A000F70198C703A7C80298CB03A7080523AC78
:1024B0000700D8CB03A80803034708006318671C6C
:1024C0004287050783460700B3050741E38B66FE95
:1024D0008981C205C181239EB700850E93870702BB
:1024E000638E121B83264E00D8422322EE00E31F88
:1024F000EFF80327CE002322EE0049BF83274E00CA
:10250000130F8E00DC432322FE006389E71B83A2A6
:10251000C700DC43AA95814E2322FE00894F130396
:10252000500A6305FF0683A8C7009387480323A0CA
:102530001501DCC183A7880423A6F5019CC583A7E8
:10254000C8029CC983A7080523AC0500DCC903A801
:1025500008038347080063976710C287850783C60F
:10256000070033870741E38B66FE098342074183F7
:10257000239EE500850E93850502638D120F832748
:102580004E00DC432322FE00E31FFFF88327CE002A
:102590002322FE0049BF83274E0A17EF0100130FC5
:1025A000AF28DC4317E70100232EF7266382E713E9
:1025B00083A2C700DC43AA95814E17E701002323BD
:1025C000F726914F1303500A6387E70783A8C700D4
:1025D0009387480323A01501DCC183A7880423A6A1
:1025E000F5019CC583A7C8029CC983A7080523AC35
:1025F0000500DCC903A80803834708006394670447
:10260000C287850783C6070033870741E38B66FED1
:10261000098342074183239EE500850E93850502C9
:10262000638A120383274E0ADC4317E70100232B3A
:10263000F71EE39DE7F98327CE0A17E7010023235E
:10264000F71E69B70147239EE500850E93850502B5
:10265000E39A12FD83274E0B769493155400E38E74
:1026600007CC91B30147239EE500850E93850502B3
:10267000E39712F117EE0100130E8E1083270E0A56
:10268000769493155400E38D07D031B78145239E8E
:10269000B700850E93870702E39612E597E70100DE
:1026A000938787F303AE070076949315540083272E
:1026B0000E00E38F07CC99B58145BDB38327CE00CB
:1026C0002322FE00A9B58326CE002322DE0055B3C7
:1026D0008327CE0A17E701002326F714D1BD8327ED
:1026E0000E0C17E701002329F714D9B9797126D206
:1026F0004AD04ECE52CC56CA5AC85EC606D622D44E
:1027000097E90100938989EA17E90100130949074C
:1027100017EA0100130A0AEB97EA0100938A4AECD0
:1027200097EB0100938BCBEA97E40100938484EA52
:10273000054B21A883A709000324090A850717E789
:1027400001002325F7E6C93011E89C40E5F783270F
:102750000900E37CFBFEEFD07FCBC5BF7370043074
:1027600083270A00B9E38327C90AC0471305440039
:10277000EFD01FE083A70B00FD1717E70100232907
:10278000F7E49C40FD1717E701002325F7E48327B2
:102790000A0089C783A70A00FC4385E30858EF10A5
:1027A00050042285EF10F0034DB703A70A0083A75A
:1027B0000A007C4385077CC37DB703A70A0083A674
:1027C0000A007C43FD177CC3FC42E9FB73600430C4
:1027D000F1B797E70100938767DD9C43DDE741117F
:1027E00006C622C426C297E7010023A907DC17E723
:1027F00001001307E7DE1C43B7A6A5A59386565A2A
:102800009C5B8C43639BD500D0436318B600944710
:102810006395C600DC476388D70008430C43938563
:102820004503EF20607417E701001307E7D914434D
:1028300017E401001304C4F411A81C43A9CF1C43DE
:10284000FD1797E6010023A1F6D8144393972600BD
:10285000B6978A07A2979C43EDD3084393172500A8
:10286000AA978A073307F4005443A107A297C442EA
:1028700044C36385F402DC44B240224417E70100FC
:102880002320F7D6924441018280854717E7010053
:102890002326F7D282807370043001A0C440D14552
:1028A000EF604013229544C1F9B701114AC806CE22
:1028B00022CC26CA4EC62A897370043097E40100E0
:1028C000938444D09C4017E40100130464D1D9E7F9
:1028D0006314090003290400930949004E85EFD0D1
:1028E0003FC98327890289C713058901EFD05FC8D3
:1028F000CE8517E501001305E5F3EFD0FFC29C403C
:1029000081C71C40FC43ADE31C40638B27079C4000
:102910009DCF737004309C40C1EB97E70100938713
:10292000E7CB9843184325EBFD5717E70100232118
:10293000F7C89C4089CF1C40FC4391CB1840144001
:102940007C43FD177CC3FC4299E373600430F24082
:102950006244D2444249B2490561828018401C4019
:102960007C4385077CC3ADB7184014407C43FD17FA
:102970007CC3FC42D1FB736004301C40E39927F90F
:102980009C40A1C397E70100938747C29C43ADCB0E
:102990007370043001A09C43DC47DC47DC4317E73D
:1029A00001002327F7C071B718401C407C438507FE
:1029B0007CC397E70100938767C2984318432DD7DC
:1029C000D9BF97E701009387A7C017E70100130756
:1029D00027DB9C430327470B631DF700F24062444B
:1029E00097E7010023AE07BED2444249B2490561D0
:1029F00082806244F240D2444249B2490561D1BB6F
:102A00006244F240D2444249B24905616FD01FA0EE
:102A10003DC9411126C297E40100938464BC4AC0B9
:102A20002E898C4006C622C4E105EFD07FB18840D4
:102A30001105EFD0FFB3FD57630AF90497E70100D2
:102A40009387C7B8804398409C434A9440C3636CC3
:102A5000F40497E70100938767B888438C40910599
:102A6000EFD01FAE97E70100938787B49C4363764E
:102A7000F40097E7010023AD87B2B24022449244AC
:102A80000249410182807370043001A08C402244CD
:102A9000B2409244024917E501001305A5D99105FA
:102AA00041016FD07FA897E701009387E7B2884381
:102AB00022448C40B24092440249910541016FD0BA
:102AC0003FA811C997E70100938747AE9C4399E758
:102AD0007370043001A07370043001A0411126C24C
:102AE00097E401009384C4AF9840AE878C40B7064A
:102AF0000080D58F06C622C41CCFE1053284EFD0FA
:102B0000BFA288401105EFD0BFA6FD57630EF400A9
:102B100097E70100938787AB8843B24092442295A0
:102B2000224441016FE08FF58C402244B240924430
:102B300017E50100130505D0910541016FD0DF9E17
:102B400025CD411126C297E40100938464A94AC0AF
:102B50002E898C4006C622C4E1053284EFD0DF9C6A
:102B600088401105EFD0DFA08547630AF40497E79A
:102B700001009387A7A5804398409C434A9440C393
:102B8000636CF40497E70100938747A588438C4062
:102B90009105EFD0FF9A97E70100938767A19C43C7
:102BA0006376F40097E7010023A487A0B240224493
:102BB00092440249410182807370043001A08C402C
:102BC0002244B2409244024917E50100130585C62C
:102BD000910541016FD05F9597E701009387C79FEB
:102BE000884322448C40B2409244024991054101FD
:102BF0006FD01F95411106C622C426C25C45C0474E
:102C000035CC930484012685EFD09F9697E7010089
:102C10009387C7999C43B5E7930444002685EFD07A
:102C20003F9597E701009387279A58549C4363F692
:102C3000E70097E7010023A9E79893172700BA97C1
:102C40008A0717E501001305A5B3A6853E95EFD0C9
:102C5000BF8D97E701009387A7989C43585401457F
:102C6000DC5763F8E700854717E701002328F7944E
:102C70000545B24022449244410182807370043081
:102C800001A0A68517E50100130545B8EFD0DF893F
:102C9000C9B797E70100938767919C4381E77370F9
:102CA000043001A0411106C622C426C2B707008025
:102CB0004045CD8F1CC12DC4EFD09F8B93044400A1
:102CC0002685EFD0FF8A97E701009387E78F585456
:102CD0009C4363F6E70097E7010023A7E78E93176D
:102CE0002700BA978A0717E50100130565A93E95E5
:102CF000A685EFD07F8397E701009387678E9C437B
:102D000058540145DC5763F8E700854717E7010091
:102D10002326F78A0545B24022449244410182802D
:102D20007370043001A011CD97E701009387C78825
:102D3000984397E70100938767899C4318C15CC15A
:102D400082807370043001A055C1D1CD411106C6F7
:102D500022C42A877370043097E80100938888861C
:102D600083A7080091CB97E7010093876787944377
:102D70009C43FC428507FCC217E301001303038553
:102D80009C4103260300FD560144638FD70217EED2
:102D90000100130E6E8203250E0003280700544322
:102DA0006305A80005446371D6023308D640054484
:102DB000637CF80003250E00918F03260300B6976D
:102DC0009CC108C350C3014483A7080081CB97E787
:102DD00001009387E7809C43FC4381EF2285B2404A
:102DE0002244410182807370043001A0737004306A
:102DF00001A0EFE0EFCEDDB7854717D70100232F05
:102E0000F77A828019C1684582800145828011C1AC
:102E10006CC5828097D701009387877C8843828026
:102E200097D701009387077A9C43054589CB97D7AD
:102E300001009387A7778843133515000605828024
:102E400031CD011126CA97D40100938464799C4046
:102E500006CE22CC4AC84EC65855DC576379F702D5
:102E60001C4D63C707009C40D4579547958F1CCDD8
:102E700093172700BA97584917E901001309499099
:102E80008A07CA97630DF7009C40DC575CD5F24077
:102E90006244D2444249B2490561828082809309EA
:102EA00045002A844E85EFD0AFEC9C4017D7010037
:102EB000130787711843DC575CD46376F70017D784
:102EC00001002323F770139527003E9562440A05FD
:102ED000F240D244CE854A95B249424905616FD04D
:102EE000AFE419CD411106C622C426C297D701000E
:102EF0009387076F80436307A4007370043001A0B9
:102F0000014582807C4881E77370043001A05454ED
:102F10003848FD177CC86383E60099C70145B24075
:102F20002244924441018280930444002685EFD0DC
:102F30002FE4284897D7010093870769984395475E
:102F4000898F48D41CCC6376A70097D7010023ADA6
:102F5000A766D145EF50102897E701009387478275
:102F60003E95A685EFD04FDC054555BF7370043004
:102F700097D70100938707659C4391CB97D70100B2
:102F80009387076698439C437C4385077CC3828074
:102F900097D70100938707639C438DC397D70100A0
:102FA000938707649843784311CB984394437C43B9
:102FB000FD177CC3FC4299E373600430828097D78D
:102FC00001009387E7619043944398439547D45613
:102FD000084E958F1CCF828097D70100938747605A
:102FE000984309C79443F84A0507F8CA8843828082
:102FF00079714AD006D622D426D24ECE2A89737051
:10300000043097D401009384E45B9C4017D4010002
:103010001304045DBDE31C40BC4F89E71C40054719
:10302000F8CFD1E19C4081C71C40FC43F1EB7370A9
:1030300004309C408DEF1C40A84F11C56304090269
:103040001C4023AC07041C4023AE07049C4081C7EE
:103050001C40FC438DEBB250225492540259F24969
:103060004561828018403C4FFD173CCFE9BF1840B6
:103070001C407C4385077CC37DBF18401C407C43BB
:1030800085077CC349BF184014407C43FD177CC3AF
:10309000FC42F1F373600430B2502254925402594E
:1030A000F2494561828008402EC61105EFD04FCC11
:1030B000B245FD576380F50697D701009387075106
:1030C00083A9070018409C43AE992322370163EC83
:1030D000F90497D701009387675088430C40910506
:1030E000EFD00FC697D701009387874C9C4363F6B8
:1030F000F90097D7010023AD374BEFD02FB11DB7A3
:10310000184014407C43FD177CC3FC428DF3736070
:10311000043031BF0C4017D501001305A57191058E
:10312000EFD08FC0D9BF97D701009387E74A884374
:103130000C409105EFD0CFC0C9B779714AD04ECEBF
:1031400006D622D426D252CC2E89B289737004308E
:1031500097D40100938404479C4017D401001304C2
:103160002448F9EF18408947784F630CF7001C405A
:103170001345F5FFB84F798DA8CF1C400547F8CF10
:10318000ADE69C4081C71C40FC43F5E373700430FE
:103190009C40B1E7638609001C40BC4F23A0F900A6
:1031A000184085470145784F630BF7001C401349D1
:1031B000F9FF0545B84F3379E90023AC27051C40DA
:1031C00023AE07049C4081C71C40FC43C1E3B250BE
:1031D000225492540259F249624A45618280184051
:1031E0001C407C4385077CC375B7084036C6110573
:1031F000EFD00FB8B246FD576385F60897D70100A8
:103200009387C73C03AA070018409C43369A2322A1
:1032100047016363FA0897D701009387273C8843E7
:103220000C409105EFD0CFB197D701009387473875
:103230009C436370FA0697D7010023AB473791A8E8
:1032400018401C407C4385077CC329BF18401440AC
:103250007C43FD177CC3FC42BDFB73600430B2505D
:10326000225492540259F249624A456182801840C0
:1032700014407C43FD177CC3FC4289FB736004301F
:1032800031B70C4017D501001305C55A9105EFD091
:10329000AFA9EFD0AF97F5B597D701009387C733A4
:1032A00088430C409105EFD0AFA9E5B751C141115A
:1032B00006C622C426C24AC07370043097D40100E7
:1032C000938444309C40B9EB99C23C4D9CC2B28778
:1032D0008946704D74CD2E872A846386D70663FC99
:1032E000F6048D456387B70091456395B700630089
:1032F000D60C38CC8547630FF60405449C4081CB3F
:1033000097D701009387C72D9C43FC43A9E32285EF
:10331000B2402244924402494101828097D7010081
:103320009387072C98439C437C4385077CC369BFE4
:103330007370043001A08546E39ED7FA3C4D33E715
:10334000B70038CD45BF3C4D85073CCD65B7EFD0C4
:103350003FF975BF130944004A85EFD06FA197D795
:1033600001009387672648549C4363F6A70097D7CC
:10337000010023ABA724D145EF50C06597D70100CA
:10338000938707403E95CA85EFD00F9A1C5481C79A
:103390007370043001A097D70100938767249C4382
:1033A0005854DC57E3FBE7F4EFD04F86B9B701443C
:1033B000B1B739CD011122CC26CA4AC84EC652C473
:1033C00056C206CEBA89368AB2842E892A84EFD0B4
:1033D000CF8FAA8A63050A003C4C2320FA00784C60
:1033E00089477CCC6389F40263F4970C8D4663872C
:1033F000D40091466396D400630AF70A232C24056F
:103400008547631EF7061C5499CB7370043001A0E6
:103410007370043001A03C4C85073CCCD5B797D7DE
:1034200001009387A7189C43ADEB930444002685C5
:10343000EFD00F9497D701009387071948549C4306
:1034400063F6A70097D7010023A0A718D145EF5036
:10345000605897D701009387A732A6853E95EFD095
:10346000AF8C97D701009387A7179C435854DC571C
:1034700063F7E70063850900854723A0F900054449
:103480005685EFD02F842285F2406244D2444249CF
:10349000B249224A924A056182809305840117D578
:1034A00001001305A536EFD02F8865BF0144C9BFC1
:1034B0008547E397F4F43C4C33E92701232C24059A
:1034C00081B74DC1011122CC26CA2A844EC606CE30
:1034D0004AC8AE84EFC07FFF8947744C7CCC3C4C1B
:1034E0000547AA8985073CCC6395E6061C5481C72D
:1034F0007370043001A097D701009387270B9C437A
:10350000ADE7130944004A85EFD08F8697D70100B5
:103510009387870B48549C4363F6A70097D7010015
:1035200023A4A70AD145EF50E04A97D7010093871B
:103530002725CA853E95EFC03FFF97D701009387A7
:10354000270A9C435854DC5763F5E70099C0854728
:103550009CC06244F240D24442494E85B249056162
:103560006FC05FF67370043001A09305840117D516
:1035700001001305A529EFC03FFBC1B7AA8729C5E4
:103580007370043017D701001307C70314439DE27B
:10359000F04F894601456315D60023AE0704054563
:1035A0001C4381CB97D701009387870398437843C7
:1035B00015E3828097D6010093868602904294425A
:1035C0007442850674C2E9B797D701009387470113
:1035D0009C437DB7984394437C43FD177CC3FC42D6
:1035E000E9FB7360043082805D71A6C2CAC052DC00
:1035F00056DA5AD85ED686C6A2C44EDE62D466D2E9
:103600006AD017D901001309A9FE17DB0100130BBB
:103610006BFD97D40100938424FD97DA0100938A0F
:10362000EAFC054AA54B832709009843630107126A
:10363000DC4783A90700EFE02FF8EFE0EFF88327DE
:103640000B002A8C6362F50A97D7010023ACA7F818
:1036500001466370351B8840B3858941EFD0FFB4C4
:10366000EFE09F9A630105128840814601462C00D5
:10367000EFD00FE34DD9A247E3C807FEC24983A7A5
:10368000490189C713854900EFC09FEEEFE0CFF3F2
:1036900083270B002A8C636DF508A24717D701001A
:1036A000232287F5E3E2FBFCB317FA0013F70721A7
:1036B000631A071613F7770C6318071E93F70702B0
:1036C000C5D74E85EF00F01145B7DC47C04783AC46
:1036D0000700930944004E85EFC09FE95C502285A6
:1036E00082975C4C6384470B83270900984371FFE2
:1036F00003A70A0097D6010023A686EF97D60100FC
:1037000023A6F6EE97D7010023A4E7EEEFE0DF8FC4
:10371000A1BFDC47C04703AD0700930C440066859A
:10372000EFC01FE55C50228582975C4C6386470999
:1037300083270900984371FF03A70A0097D6010069
:1037400023A6F6EA97D7010023A4E7EAB9B7EFE08A
:10375000AFE6EFE06FE783270B002A8CE366F5F80E
:1037600083A70A00884081499043B385894117D7D0
:103770000100232987E713361600EFD01FA3EFE0DF
:10378000BF88E31305EEEFC07FC8F9BD1C4CCE85A2
:10379000E69763E9FC049C4089CF02CA66CC22CE3E
:1037A000EFF00FE88840814601464C08EFC03FFF2C
:1037B00005FD7370043001A01C4CE685EA97636C2C
:1037C000FD049C4089CF02CA6ACC22CEEFF04FE5BF
:1037D0008840814601464C08EFC07FFC31F9737088
:1037E000043001A0032509005CC000C8EFC05FD50C
:1037F000E5BDEFE07F8183270900DC47C047930CDC
:1038000044006685EFC0DFD65C4C638F47035C5095
:103810002285829791BD032509005CC000C8EFC0D6
:103820003FD239B7B24723ACF900A5CFE29723A224
:10383000F90023A8390193854900636FFC0403A5AF
:103840000A00EFC0FFCF0DB51C4C00C83387F9004C
:1038500058C0636DEC02330C3C416363FC029C4036
:1038600089CF02CA4ECC22CEEFF08FDB8840814652
:1038700001464C08EFC0BFF259F97370043001A043
:1038800003A50A00E685EFC0BFCB51B703250900A9
:10389000E685EFC0FFCAA5BF03250900EFC05FCAD8
:1038A000E1B37370043001A0B24783A6890123A855
:1038B00039013387D70023A2E9006364EC04B3071E
:1038C000FC4063EBD70483A749024E85829783A708
:1038D000C901E39B47D983A68901B2479840B697AF
:1038E00011CF02CA3ECC4ECEEFF08FD38840814636
:1038F00001464C08EFC0BFEAE31805D673700430E8
:1039000001A06374FC00E370F7FC032509009385B4
:103910004900EFC0FFC289BB03A50A009385490097
:10392000EFC01FC291B3411122C406C626C24AC0CD
:1039300017D40100130444CBEFF04FE31C4095CBA8
:10394000EFF00FE51C409DC38148014881470947BE
:1039500081461306004097D501009385A5AD170554
:1039600000001305A5C8EFD07F9939E973700430C2
:1039700001A017D90100130929ED4A85EFC03FB90D
:1039800097D40100938484ED2685EFC05FB801468B
:10399000B145114597D7010023AC27C597D7010042
:1039A00023A697C4EFC09FD217D70100232EA7C22A
:1039B00011CD97D50100938565A7EFD0CFF349B717
:1039C000B240224492440249410182807370043023
:1039D00001A0A5C9797156CAAA8A1305C00222D4CA
:1039E00026D24AD04ECE52CC06D65AC85EC63A89A6
:1039F000B689328AAE84E9212A8405C9EFF00FD74F
:103A000097D70100938747BE9C439DCFEFF04FD8D7
:103A1000130544002320540104CC232E4401232009
:103A2000340323222403EFC0DFAF2285B250225497
:103A300092540259F249624AD24A424BB24B456112
:103A400082807370043001A097DB0100938BCBDF81
:103A50005E85EFC0DFAB17DB0100130B2BE05A854F
:103A6000EFC0FFAA0146B145114597D7010023A138
:103A700077B997D7010023AB67B7EFC03FC517D71A
:103A800001002323A7B601C997D501009385059AA4
:103A9000EFD06FE6A5BF7370043001A039C50111E6
:103AA00022CC06CE26CA17D401001304E4B383281F
:103AB00004002A88014563850802BA842EC236872D
:103AC00032C442C6954663C5B602EFF06FB589476A
:103AD000630BF5020840814601464C00EFC03FCC25
:103AE000F2406244D244056182807370043001A0C8
:103AF0004C0081463A864685EFC0BFFFF2406244E3
:103B0000D244056182800840814626864C00EFC081
:103B10001FC9F9B719C1084182807370043001A030
:103B200001E57370043001A0411106C622C42A8445
:103B3000EFF0CFC348483334A000EFF06FC52285C3
:103B4000B24022444101828001E57370043001A03B
:103B5000411122C42A8406C6EFF04FC10050EFF095
:103B60002FC3B240228522444101828001E5737057
:103B7000043001A0411122C426C22E84AA8406C6A4
:103B8000EFF0CFBE80D02244B240924441016FF0AA
:103B90002FC04111714522C406C61D262A8411C5B5
:103BA000232005001105EFC09F962285B2402244D4
:103BB0004101828001CDB70700FFED8F81C773708F
:103BC000043001A099E57370043001A073700430D3
:103BD00001A0011122CC4AC84EC652C456C206CE1C
:103BE00026CABA893689B28A2E842A8AEFF04FA370
:103BF00011E5638509007370043001A0EFE0CF9BED
:103C000083240A00B37794006316090295C763877B
:103C10000A009347F4FFE58F2320FA00EFE0CFBEC0
:103C2000F240624426854249D244B249224A924A2D
:103C300005618280E30DF4FCE38209FEB335500197
:103C4000E20563050900B7070004DD8D4E86C18DCE
:103C500013054A00EFE0FFE6EFE00FBB19E1EFC00C
:103C6000EFFAEFF0CFB593176500AA8963D8070084
:103C7000B7040001FD14B3F499005DB7EFF00FAF86
:103C800083290A00B3773401631E090089CB638856
:103C90000A009347F4FFB3F737012320FA00EFF04F
:103CA0002FAFF9B7E31DF4FEDDB701C9B70700FF79
:103CB000ED8F99C77370043001A07370043001A0B8
:103CC000411122C42A8406C626C24AC02E89EFF0BA
:103CD000EFA904409345F9FFB3F795001CC0EFF03E
:103CE0002FABB24022442685024992444101828092
:103CF000411122C42A8406C6EFC02FFD0040EFC048
:103D00006FFCB240228522444101828009C93707F5
:103D100000FFB3F7E50099C77370043001A073701A
:103D2000043001A06F40505DB70700FFF18F81C7DD
:103D30007370043001A001E67370043001A001111A
:103D400022CC4AC84EC652C406CE26CA3689AE898F
:103D50002A8A3284EFF0CF8C21E163050900737069
:103D6000043001A0EFE04F8583240A00CE85528500
:103D7000B3E49900613FB37794006307F4068324AA
:103D80000A00EFE06FA8F240624426854249D2441F
:103D9000B249224A05618280EFE00F8283240A0043
:103DA000CE855285B3E434019537B3F78400638D33
:103DB0008702E30609FCB70500054A86C18D130595
:103DC0004A00EFE01FD0EFE02FA419E1EFC00FE4AD
:103DD000EFF0EF9E93176500AA8463DF0700B70733
:103DE0000001FD17FD8C45B783270A001344F4FF3B
:103DF000E18F2320FA0071B7EFF04F9783240A0078
:103E0000B3779400639787009347F4FFE58F2320EF
:103E1000FA00EFF0EF97E1B7411122C406C62A84F9
:103E200026C2EFD07FF95C4085C308489304C400E4
:103E30006316950015A0084863009502B7050002B7
:103E4000EFE03FE55C40E5FB2285612A2244B24079
:103E5000924441016FE04F9B7370043001A009C987
:103E6000370700FFB3F7E50099C77370043001A06E
:103E70007370043001A06F40304801C9B70700FFDC
:103E8000ED8F99C77370043001A07370043001A0E6
:103E9000411122C426C206C62A84AE84EFF00F8DDB
:103EA000184093C7F4FFF98F1CC02244B2409244DB
:103EB00041016FF0EF8D19C1084D8280014582806C
:103EC000411122C406C62A84EFD01FEF97C7010014
:103ED000938747729C43A1EBE56717D7010013074F
:103EE0006799F11797C6010023ACE67017C7010068
:103EF0002326F77017D701002320F79897C70100F2
:103F00009387876F17D701002326F796854717C732
:103F100001002329076E17C70100232F076C17C75D
:103F200001002329F76C19E8EFE00F8EEF10400332
:103F300001442285B240224441018280130584005D
:103F400093773500C1EFE5671307F5FFE917E3ED58
:103F5000E7FC97C601009386A66A9C4229A0984375
:103F600011C7BE86BA87D843E36BA7FE17C7010007
:103F700013078768E38AE7FA98434146138487006A
:103F800098C2D843B306A7406378D6023388A70007
:103F90002322D800C8C38325480097C60100938612
:103FA000266611A0BA8698425043E36DB6FE2320E0
:103FB000E80023A00601D84397C701009387077440
:103FC0009C43998F17C70100232AF772EFE0CF8334
:103FD00031DC2285B2402244410182807199110571
:103FE0009DB729C9411122C406C62A84EFD0DFDC5F
:103FF000930584FF0326C4FF17C70100130747601A
:1040000011A03E871C43D443E3EDC6FE232CF4FEEF
:104010000CC397C701009387676E98438327C4FF3B
:104020002244B240BA9717C701002329F76C410117
:104030006FD09FFD828097C701009387276C8843CC
:10404000828082803367B5000D8BAA871DE79308B5
:10405000D6FFAA982A87AE866371150303A80600C7
:1040600011079106232E07FFE36A17FF9347F5FF19
:10407000C697F19B9107BE95AA972A9663F3C70A44
:104080009386450013884700B3B6D70033B80501BF
:1040900033E7F50093C61600134818000D8BB3E6FE
:1040A000060113371700758F330EF64093861700FD
:1040B00029CF1337AE0031EB13532E002E88BE8666
:1040C0000147832808000507110823A0160191065F
:1040D000E36967FE1377CEFFBA95BA976302EE04E1
:1040E00083C60500138717002380D700637AC702B1
:1040F00083C6150013872700A380D7006372C70209
:1041000003C725002381E7008280B307F640AE97FE
:10411000850503C7F5FF8506238FE6FEE39AF5FEC6
:1041200082808280B367C5008D8BB308C500E9C368
:104130006371150FB307A0408D8B13873700954629
:1041400093F5F50F130815003383A8407D166373AC
:10415000D70015476363E60CD5CF2300B5000547AC
:10416000638DE700A300B5000D4713082500639693
:10417000E700130835002301B500139685004D8E26
:1041800013970501518F3303F34093968501D98E20
:1041900013562300AA97014794C305079107E36DBF
:1041A000C7FE1377C3FFB307E8006307E306238066
:1041B000B70013871700637C1703A380B70013872A
:1041C0002700637617032381B700138737006370D6
:1041D0001703A381B70013874700637A170123826F
:1041E000B7001387570063741701A382B70082805A
:1041F00093F5F50F13978500D98D139705014D8F12
:10420000E37715FFAA87910723AEE7FEE3ED17FFDB
:10421000828082802A8895B78280AA8749BF834797
:1042200005002A8799C7050583470500EDFF198D0D
:1042300082800145828005058347F5FF850503C718
:10424000F5FF91C7E389E7FE3385E7408280814728
:10425000E5BFAA87850503C7F5FF8507A38FE7FE9E
:1042600075FB828083460500930700026397F60082
:10427000050583460500E38DF6FE938756FD93F70B
:10428000D70F85C7AA87814585CE01458507138647
:1042900006FD1317250083C607003A9506053295DB
:1042A000F5F699C13305A0408280938536FD83469B
:1042B000150093B5150093071500E1FA0145D5B730
:1042C000014582809C412380A7009C4185079CC1B9
:1042D000828097C60100938626339C4217570300BD
:1042E0001307475A13861700BA972380A70097C56C
:1042F000010023ABC530A9476308F500930700040C
:104300006305F6000145828075DE370610F005076B
:104310008347F7FF2320F6F09C42FD1797C5010065
:1043200023A4F52EEDF7014582804D7123229114CF
:1043300023202115232A511323248113232611140A
:1043400023248114232E3113232C4113232861139A
:1043500023267113232291132320A113232EB1119D
:10436000AA842E8932C6130C5002A54A834709003D
:1043700063808703B9CB804011A0A1CB2300F40058
:1043800080400509050480C083470900E39787FF43
:104390000346190093081900C686130D0002FD5943
:1043A0007D5A0148130550059307D6FD93F7F70F83
:1043B000138916006363F52A17C70100130787C422
:1043C0008A07BA979C43BA9782878320C114032433
:1043D000811483244114032901148329C113032A5E
:1043E0008113832A4113032B0113832BC112032C46
:1043F0008112832C4112032D0112832DC111716191
:104400008280A14C02C4854763D50715B24780401E
:10441000938B770093F68BFF03AB060083A94600CE
:10442000938786003EC6668681465A85CE85EF1004
:10443000B0782AC8814763853723930D4101854BA6
:10444000668681465A85CE85EF105019814666866C
:104450002A8BAE89EF105076A24723A0AD00938639
:104460001B00910D63843701B68BD9BFE37E9BFFA0
:1044700063DD4601A2872380A70180407D1A930750
:1044800014009CC03E84E3C846FF93962B001C0892
:10449000BE9631A8938777052300F4008040FD1B6A
:1044A00093871B00050480C0F116E351F0EC9C4299
:1044B000E3E2FAFE93870703C5B79C409306000327
:1044C00032472380D7009C4093064700C14C138697
:1044D000170090C013068007A380C700804002C465
:1044E000BA87050480C003AB0700814936C625BFE3
:1044F000B24783AC0700938B470063840C1C635F57
:1045000040199307D0026319FD1683C70C0085C3B9
:1045100063DC09189440850C7D1A2380F6008040E6
:10452000050480C083C70C00E5F7635D400180404F
:10453000930700022300F40080407D1A050480C028
:10454000E31A0AFE5EC61DB502C48547A94CE3CF37
:1045500007EBB24780409386470071B703C6160049
:10456000CA8699B59C40930650022380D7008040AC
:10457000050480C0E5BBC14C02C471B5B24703C697
:104580001600CA8683A9070091073EC6E35E0AE0CB
:104590004E8AFD5911BD03C61600130DD002CA86FE
:1045A00021B59347FAFFFD8703C61600337AFA0058
:1045B000CA86DDBB03C61600130D0003CA86EDB321
:1045C00083C51600930906FDCA86938705FD2E86CE
:1045D000E3EEFAFA93972900BE9985068609AE990B
:1045E00083C50600938909FD938705FD2E86E3F3B5
:1045F000FAFE69BF32479C40144311073AC6238034
:10460000D7008040050480C095B3854763D3070B6E
:10461000B24793867700E19A938786003EC683A9C6
:1046200046009C4263DC090A94401306D002B3079B
:10463000F0402380C6008040B336F000B30930411B
:10464000050480C03E8BB389D940A94C02C4E1BBAC
:1046500003C616000508CA8681BB9C40468921B75F
:10466000E37D9BDD8547814B8546E3C547E131BD51
:1046700097CC0100938C8CDCCE856685EF10401EB4
:10468000330AAA40635C400180402300A4018040BB
:104690007D1A050480C0E31A0AFE014A83C70C0094
:1046A000E38207EAE3C809E6FD197D57E394E9E6EA
:1046B000ADBDB247938647009C4336C693D9F741B8
:1046C00095B7635640019307D002E313FDFA97CCE8
:1046D0000100938CACD6930780021DBD3E8BA94C84
:1046E00002C4804089B34D71232E3113B7090040B5
:1046F0009387F9FF2324811423229114232C41133F
:10470000232A511323261114232021152328611352
:104710002326711323248113232291132320A11311
:10472000232EB1112A8A2EC417C401001304C4ED2C
:10473000975A0300938A0A1597C40100938404A230
:104740003EC693055002294513080004B70610F031
:1047500083470A006386B704C1C71840050A1306D9
:104760001700569797C8010023A0C8EA2300F70056
:104770006382A706E31E06FD175703001307871081
:1047800005078347F7FF23A0F6F01C40FD1717C667
:104790000100232BF6E6EDF783470A00E39EB7FA04
:1047A00083461A0013051A002A87930B00027D5BCB
:1047B0007D5C014893055005A5489387D6FD93F786
:1047C000F70F130A170063E7F5348A07A6979C438F
:1047D000A6978287175703001307C70A55F28DBFA4
:1047E0008320C11403248114832441140329011458
:1047F0008329C113032A8113832A4113032B011335
:10480000832BC112032C8112832C4112032D011220
:10481000832DC11171618280A14C014D854763DBFD
:104820000719A2479D07E19B83AD070003AB470033
:10483000138787003AC4668681466E85DA85EF1055
:10484000B0372AC863066D3513094101854966866C
:1048500081466E85DA85EF10605866868146AA8D9E
:104860002E8BEF1070352320A90085091109E31064
:104870006DFFE3FE9DFD13060004B70610F063D143
:1048800089031C4013871700D69797C5010023ADF5
:10489000E5D623807701630CC7047D1CE3C389FF41
:1048A000B2476800A548B386F9008A061C08BE9680
:1048B000294813030004370610F0E384A6E89C425D
:1048C0009305000363F4F800930570051840AE9754
:1048D00093051700569717CE01002327BED2230059
:1048E000F7006380072B638C6526F116F9B717571D
:1048F0000300130727F905078347F7FF23A0F6F006
:104900001C40FD1797C5010023A0F5D0EDF77D1CD5
:1049100071B71C40130600041387170097C50100E8
:1049200023A4E5CEB386FA00930500032380B600E6
:104930006300C73E890797C6010023A7F6CC5697A8
:10494000930680072300D70017570300130787F348
:10495000B70610F0639EC70005078347F7FF23A043
:10496000F6F01C40FD1717C60100232FF6C8EDF71F
:10497000A247C14C014D91072247014B832D0700EF
:104980003EC455BDA24783AC070013894700638F1F
:104990000C3A635480219307D002639EFB2E03C719
:1049A0000C00BA856310072025AC8547A94C014D42
:1049B000E3C907E7A2479107C1B7A247834617009B
:1049C000528703AB070091073EC4E3580CDE5A8CB4
:1049D0007D5BE5B383461700930BD0025287F1BB92
:1049E0009347FCFFFD8783461700337CFC0052870A
:1049F000E9B383461700930B000352877DBB034640
:104A00001700138B06FD5287930706FDB286E3EE6F
:104A1000F8FA93172B00DA9705078607B297034633
:104A20000700138B07FD930706FDB286E3F3F8FE3C
:104A300069BFA2451C402946984193861700D69726
:104A400017C501002322D5BC2380E7001389450048
:104A50006301C72A930700046387F6204AC4D5B1CF
:104A6000854763DF0729A24713877700619B930778
:104A700087003EC4032B47001C43635B0B30184088
:104A8000130600049306170097C5010023AED5B6A0
:104A900056979305D0022300B7006388C62CB3074E
:104AA000F0403337F000330B6041BE8D330BEB40E9
:104AB000A94C014D49B38346170005085287F5B943
:104AC000834617005287D5B91C409306000413870C
:104AD000170017C601002329E6B2D6971306500225
:104AE0002380C700E31FD7C417570300130787D9D4
:104AF000B70610F005078347F7FF23A0F6F01C4028
:104B0000FD1717C601002321F6B0EDF71DB9C14C02
:104B1000014D29B31C40930600042A8A138717000D
:104B200017C601002322E6AED69713065002238053
:104B3000C700E318D7C0175703001307A7D4B70659
:104B400010F005078347F7FF23A0F6F01C40FD1780
:104B500017C60100232AF6AAEDF72A8ADDB61757F1
:104B60000300130727D205078347F7FF2320F6F03A
:104B70001C40FD1797C5010023A8F5A8EDF7F11615
:104B80002DBB175703001307E7CFF1FDF11635B31F
:104B9000E3FC9DCB8549C5B1014C03C70C00BA8528
:104BA000E30E07EAFD58294513080004B70610F084
:104BB00063570B0A1C4013861700D69717C30100D2
:104BC0002324C3A42380E7006384A50663040609A5
:104BD000850C03C70C007D1CBA8579FBE35080E986
:104BE0001C409305000213060004B70610F021A034
:104BF0007D1CE3050CE613871700D6972380B700CA
:104C000017C501002322E5A0BA87E313C7FE175793
:104C10000300130727C705078347F7FF23A0F6F014
:104C20001C40FD1717C501002320F59EEDF7C9B7FD
:104C300017570300130707C541DE05078347F7FF32
:104C400023A0F6F01C40FD1717C60100232EF69A8C
:104C5000EDF7BDBF175703001307C7C2F9BF7D1B90
:104C6000E31A1BF5A5BF175703001307A7C1B70623
:104C700010F005078347F7FF23A0F6F01C40FD174F
:104C800017C601002322F698EDF74AC45DBC97BC15
:104C90000100938CAC7ADA856685EF00703C330CAA
:104CA000AC40E35C80EF1C4013060004B70610F034
:104CB00021A07D1CE3020CEE13871700D6972380FA
:104CC000770197C5010023A1E594BA87E313C7FED6
:104CD00017570300130707BB05078347F7FF23A0F8
:104CE000F6F01C40FD1797C5010023AFF590EDF7D6
:104CF000C9B7175703001307E7B8B5FA4AC491B408
:104D0000A247138747009C433AC413DBF741B5B36E
:104D100017570300130707B7B70610F005078347B7
:104D2000F7FF23A0F6F01C40FD1717C60100232D46
:104D3000F68CEDF7854717C701002327F78C9307FB
:104D4000800717570300230FF7B21DB16356800188
:104D50009307D002E39DFBF297BC0100938C0C6E8D
:104D6000130780029305800235BD97560300938692
:104D700066B1370610F0850603C7F6FF2320E6F07C
:104D800018407D1797C5010023A0E5886DF701BB8A
:104D9000BE8DA94C014D45B4B70710F023A0A7F272
:104DA00001A03971130341022ED29A8506CE32D466
:104DB00036D63AD83EDA42DC46DE1AC62D32F2400A
:104DC0000145216182805D711303810322D42AC6CB
:104DD00032DC2A841A86680006D6BEC236DEBAC025
:104DE000C2C4C6C61ACEEFF04FD4B2472380070024
:104DF0003245B250018D225461618280B70710F0B4
:104E000083A647F403A607F403A747F4E31AD7FEE3
:104E10008566938606FAB29633B6C600B305E600F9
:104E200023A4D7F423A6B7F48280B70710F003A712
:104E300047F403A607F483A647F4E31AD7FE856672
:104E4000938606FAB29633B6C60023A4D7F4B30508
:104E5000E60023A6B7F49307000873A047308280CA
:104E6000411122C406C697B701009387677A17B429
:104E700001001304A47998431C401306F07C9306A8
:104E800047069387470697B5010023A3D57897B5C2
:104E9000010023ADF5766346D600B24022444101BD
:104EA00082801307478997B7010023A3E776EF00B5
:104EB000D01385476310F502184085679387F7760E
:104EC0000145E3DCE7FCEFF03FED2244B240410155
:104ED0006FC09FED17B501001305C556EFF07FECCD
:104EE0000945EFF07FEB2244B24041016FC0DFEB98
:104EF00017B50100130585566FF0BFEA17B501001D
:104F0000130545566FF0FFE9411122C426C206C6BB
:104F1000856417B401001304645593878438010035
:104F2000FD17F5FF2285EFF0DFE7C5BF01456F00F4
:104F3000F000411106C6EF00500B0547814763168C
:104F4000E500B2403E854101828017B5010013059E
:104F5000654FEFF01FE5B24089473E8541018280F1
:104F60007370043001A082807370043001A097B781
:104F700001009387A76A9843DC4359713AD43ED61F
:104F800097B701009387076ADAC8DEC603AB07004C
:104F900083AB470097B7010093874769D2CCD6CA45
:104FA00003AA070083AA470097B701009387876881
:104FB000CAD0CECE03A9070083A94700E2C4E6C247
:104FC000EAC06EDE86D6A2D4A6D2AA8D814C17BCCA
:104FD0000100130CAC66370D00805AC45EC652C87F
:104FE00056CA4ACC4ECE2245B2454246D2466244CB
:104FF000F244EF10700C2286A686EF20F02C2AD007
:105000002ED2025592552256B256EF30E01A014682
:105010008146EF20B01B6349050202559255225686
:10502000B256EF30601903260C0083264C00EF20A7
:10503000300A3325A00019E5E3910CFA8547239047
:10504000FD0061BF854C51BF8257125822563E87E2
:10505000B3470D01B2563A85BE85E1B7597197B78E
:1050600001009387275EDAC803AB0700DEC683AB77
:10507000470097B701009387675DD2CC03AA07006A
:105080005AC4D6CA83AA470097B701009387875CA2
:105090005EC6CAD003A9070052C8CECE83A9470076
:1050A00056CA4ACC4ECE2247B2474246D246A2D436
:1050B000A6D26244F2446EDEBE85AA8D3A8586D6BB
:1050C000E2C4E6C2EAC0EF10B07F2286A686EF20D7
:1050D000B01F2AD42ED6814C17BC0100130C0C56DD
:1050E000370D00805AC45EC652C856CA4ACC4ECE4E
:1050F0002245B2454246D2466244F244EF10507C0B
:105100002286A686EF20501C2AD02ED20255925518
:105110002256B256EF30400A01468146EF20100B6E
:1051200063490502025592552256B256EF30C00827
:1051300003260C0083264C00EF2080793325A00045
:1051400019E5E3910CFA85472390FD0061BF854C7A
:1051500051BF8257125822563E87B3470D01B256AF
:105160003A85BE85E1B775712AD61305000522C5BB
:1051700026C34AC1CEDED2DCD6DADAD8DED6E2D415
:10518000E6D2EAD0EECE06C7EFE09FD397B7010094
:105190009387C74C03AB070083AB470097B7010069
:1051A0009387474C03AA070083AA470097B70100DB
:1051B0009387C74B03A9070083A9470097B701004E
:1051C0009387474B8043C44397B701009387074BAE
:1051D00003A847009C432A8C42C63EC497B70100EF
:1051E0009387474A03A847009C43814C42CA3EC864
:1051F00097B701009387874903A847009C4342CE95
:105200003ECC97B701009387E74803A847009C432B
:1052100042D23ED097B701009387474803AD0700BD
:1052200083AD470002DC02DE82C082C223200C0074
:1052300023220C006255F25501468146EF10C067EB
:105240002ADC2EDE23246C0123267C016255F255D4
:105250005A86DE86EF1040662ADC2EDE23284C01BB
:10526000232A5C016255F2555286D686EF10C0643F
:105270002ADC2EDE232C2C01232E3C016255F25514
:105280004A86CE86EF1040632ADC2EDE23208C0275
:1052900023229C026255F2552286A686EF10C06139
:1052A00022462ADCB2462EDE2324CC022326DC0250
:1052B0006255F255EF10406042462ADCD2462EDE9F
:1052C0002328CC02232ADC026255F255EF10C05E7F
:1052D00062462ADCF2462EDE232CCC02232EDC0290
:1052E0006255F255EF10405D02562ADC92562EDED2
:1052F0002320CC042322DC046255F255EF10C05B5E
:105300002ADC2EDE2324AC052326BC056255F2558B
:105310006A86EE86EF10405A2ADC2EDE03250C004A
:1053200083254C0006469646EF100059AAC0AEC22F
:1053300003258C008325CC0006469646EF10C05707
:10534000AAC0AEC203250C0183254C010646964631
:10535000EF108056AAC0AEC203258C018325CC0174
:1053600006469646EF104055AAC0AEC203250C0271
:1053700083254C0206469646EF100054AAC0AEC2E2
:1053800003258C028325CC0206469646EF10C052B8
:10539000AAC0AEC203250C0383254C0306469646DD
:1053A000EF108051AAC0AEC203258C038325CC0325
:1053B00006469646EF104050AAC0AEC203250C0424
:1053C00083254C0406469646EF10004FAAC0AEC295
:1053D00003258C048325CC0406469646EF10C04D69
:1053E000AAC0AEC26255F25506469646EF20D05C82
:1053F000AAC4AEC62645B64501468146EF20005DEB
:105400006348050297B701009387472326459043D9
:10541000B645D443EF20C04B3325A00001E9E39308
:105420000CE0B25705472390E700EDBB854CDDBB90
:1054300097B701009387072726459043B645D44385
:10544000EF20C0587D81D9BF75712AD6130500059C
:1054500022C526C34AC1CEDED2DCD6DADAD8DED601
:10546000E2D4E6D2EAD0EECE06C7EFE07FA597B74A
:1054700001009387A72303AB070083AB470097B7CF
:1054800001009387272303AA070083AA470097B741
:1054900001009387A72203A9070083A9470097B7B4
:1054A0000100938727228043C44397B70100938765
:1054B000E72103A847009C432A8C42C23EC097B70D
:1054C00001009387272103A847009C43814C42C6D3
:1054D0003EC497B701009387672003A847009C4309
:1054E00042CA3EC897B701009387C71F03A8470069
:1054F0009C4342CE3ECC97B701009387271F03A859
:1055000047009C4342D23ED097B701009387871E45
:1055100003AD070083AD470002DC02DE82C082C219
:1055200023206C0123227C016255F2555A86DE86C7
:10553000EF1080382ADC2EDE23244C0123265C0168
:105540006255F2555286D686EF1000372ADC2EDEE1
:1055500023282C01232A3C016255F2554A86CE8627
:10556000EF1080352ADC2EDE232C8C00232E9C00AD
:105570006255F2552286A686EF10003402462ADCD8
:1055800092462EDE2320CC022322DC026255F25505
:10559000EF10803222462ADCB2462EDE2324CC02D3
:1055A0002326DC026255F255EF10003142462ADC18
:1055B000D2462EDE2328CC02232ADC026255F25585
:1055C000EF10802F62462ADCF2462EDE232CCC021E
:1055D000232EDC026255F255EF10002E02562ADC13
:1055E00092562EDE2320CC042322DC046255F25591
:1055F000EF10802C2ADC2EDE2324AC052326BC05EC
:105600006255F2556A86EE86EF10002B2ADC2EDEFC
:1056100003250C0083254C0006469646EF10C02952
:10562000AAC0AEC203258C008325CC000646964650
:10563000EF108028AAC0AEC203250C0183254C01BF
:1056400006469646EF104027AAC0AEC203258C013D
:105650008325CC0106469646EF100026AAC0AEC2AE
:1056600003250C0283254C0206469646EF10C02403
:10567000AAC0AEC203258C028325CC0206469646FC
:10568000EF108023AAC0AEC203250C0383254C0370
:1056900006469646EF104022AAC0AEC203258C03F0
:1056A0008325CC0306469646EF100021AAC0AEC261
:1056B00003250C0483254C0406469646EF10C01FB4
:1056C000AAC0AEC203258C048325CC0406469646A8
:1056D000EF10801EAAC0AEC26255F255064696462D
:1056E000EF20902DAAC4AEC62645B6450146814698
:1056F000EF20C02D6348050297B70100938707F498
:1057000026459043B645D443EF20801C3325A000A6
:1057100001E9E3930CE0B25705472390E700EDBBA6
:10572000854CDDBB97B701009387C7F726459043AB
:10573000B645D443EF2080297D81D9BF411122C4D1
:105740002A872A8481480148814797B601009386B9
:1057500066EC1306004097B50100938565D21705E6
:1057600000001305058106C6EFB05FB922878148A6
:105770000148814797B601009386E6E91306004089
:1057800097B50100938545D0170500001305458D99
:10579000EFB0DFB6228781480148814797B6010004
:1057A000938686E71306004097B50100938545CEA2
:1057B00017050000130585C9EFB05FB422872244A6
:1057C000B24081480148814797B601009386E6E4DC
:1057D0001306004097B50100938505CC170500001E
:1057E0001305A59841016FB07FB197B6010083D62C
:1057F00066E2054797B701009387C7E101456397C4
:10580000E60017B70100231707E0054503D7270077
:1058100085466380E60203D74700854601456383DA
:10582000E60283D76700054701456306F702014595
:10583000828017B70100231007DE03D74700854693
:10584000E391E6FE17B70100231807DC83D7670052
:105850000547E31EF7FC97B70100239007DC828021
:10586000B305B500930705006386B70003C70700BB
:10587000631607003385A7406780000093871700F1
:105880006FF09FFE130101FB23229104232C41039F
:10589000232291032326110423248104232021059C
:1058A000232E3103232A5103232861032326710366
:1058B000232481032320A103232EB101930C05008F
:1058C000138A05009304000063DE05003305A04041
:1058D0003337A000B305B040930C0500338AE54090
:1058E0009304F0FF63DA06003306C040B337C0000C
:1058F000B306D040B386F640930A060093890600AB
:1059000013840C0013090A006396062817BB0100D4
:10591000130BCBA16370CA16B70701006372F614AC
:105920009307F00F63F4C70093098000B357360163
:10593000330BFB0083470B0013050002B3873701CD
:10594000B309F540638C0900B3153A01B3D7FC00E5
:10595000B31A360133E9B70033943C0113DB0A0173
:1059600093050B0013050900EF30000E130A050024
:1059700093050B00939B0A0113050900EF304008C3
:1059800093DB0B019305050013850B00EF308004BA
:10599000131A0A0193570401B367FA0063FAA700C8
:1059A000B387570163E6570163F4A700B387570134
:1059B0003389A74093050B0013050900EF30C00899
:1059C000130A050093050B0013050900EF3040038F
:1059D0001314040193050500131A0A0113850B0023
:1059E00013540401EF20107F33648A00637AA4000B
:1059F00033045401636654016374A40033045401F6
:105A00003304A4403354340193050000638A040036
:105A100033048040B3378000B305B040B385F54010
:105A2000130504008320C10403248104832441045A
:105A3000032901048329C103032A8103832A410323
:105A4000032B0103832BC102032C8102832C41020F
:105A5000032D0102832DC1011301010567800000A0
:105A6000B707000193090001E362F6EC9309800196
:105A70006FF0DFEB631A06009305000013051000BA
:105A8000EF201078930A0500B707010063FAFA0EB9
:105A90009307F00F63F4570193098000B3D73A01DD
:105AA000330BFB0083470B001305000233095A41F7
:105AB000B3873701B309F540E38209EAB39A3A01A3
:105AC000335BFA00B3153A01B3D7FC0093DB0A014C
:105AD00033E9B70013050B0093850B00EF20D07658
:105AE000130A050093850B00139C0A0113050B0094
:105AF000EF201071135C0C019305050013050C00D9
:105B0000EF20506D131A0A0193570901B367FA0089
:105B100033943C0163FAA700B387570163E657014A
:105B200063F4A700B3875701338BA74093850B001D
:105B300013050B00EF205071130A050093850B002D
:105B400013050B00EF20D06B9305050013050C0027
:105B5000EF20506893160901131A0A0193D6060123
:105B6000B366DA0063FAA600B386560163E656010F
:105B700063F4A600B38656013389A6406FF01FDE9A
:105B8000B707000193090001E3EAFAF093098001E5
:105B90006FF0DFF06376DA0093050A006FF01FE71D
:105BA000B707010063FAF604930BF00F33B5DB007F
:105BB0001315350033D7A60097A701009387077701
:105BC000B387E70083CB070093050002B38BAB00DC
:105BD000338B7541631C0B0263E4460163EACC001E
:105BE0003384CC40B306DA4033B98C003389264184
:105BF000930509006FF09FE1B7070001130500014D
:105C0000E3EAF6FA130580016FF0DFFAB396660156
:105C1000335D7601336DDD00B35D7A01B3156A0142
:105C200033DC7C0113540D01336CBC0013850D0073
:105C300093050400B3196601EF201061930A050073
:105C40009305040013850D0033996C01931C0D011D
:105C5000EF20105B93DC0C01130A0500930505008F
:105C600013850C00EF201057939A0A0113570C016B
:105C700033E7EA00930D0A00637EA7003307A7010C
:105C8000930DFAFF6368A7016376A700930DEAFFFF
:105C90003307A701330AA7409305040013050A0040
:105CA000EF20905A93050400930A050013050A009B
:105CB000EF201055930505001304050013850C0013
:105CC000EF20505193150C01939A0A0193D50501C9
:105CD000B3E5BA001307040063FEA500B385A50170
:105CE0001307F4FF63E8A50163F6A5001307E4FFBB
:105CF000B385A501939D0D01B70C0100B3EDED0037
:105D00001384FCFFB3F78D0033F48900338AA54078
:105D100013850700930504002326F10093DD0D0190
:105D2000EF20504B93050400930A050013850D00E6
:105D3000EF20504A13DC090193050C002324A10035
:105D400013850D00EF2010498327C10013040C00B8
:105D500093050400130C050013850700EF209047FE
:105D60008326810013D70A013305D5003307A70026
:105D70006374D700330C9C01B70701009387F7FFCA
:105D8000935507013377F70013170701B3F7FA00AC
:105D9000B3858501B307F7006366BA00631EBA00D6
:105DA000637CF90033863741B3B7C700B385A5419B
:105DB000B385F54093070600B307F9403339F9007E
:105DC000B305BA40B385254133947501B3D7670154
:105DD0003364F400B3D565016FF05FC3130101FDB7
:105DE00023229102232A5101232611022324810216
:105DF00023202103232E3101232C4101232861017B
:105E00002326710123248101232291012320A10152
:105E1000930A050093840500639E06381304060068
:105E20009309050017A901001309495063F8C51229
:105E3000B7070100138B05006378F6101307F00F06
:105E40003337C70013173700B357E6003309F9009B
:105E5000834609003387E60093060002B386E640D6
:105E6000638C0600B394D40033D7EA003314D60011
:105E7000336B9700B399DA00935A040193850A00B3
:105E800013050B00EF20503C1309050093850A0011
:105E9000931B040113050B00EF20903693DB0B01DD
:105EA000930405009305050013850B00EF20903245
:105EB0001319090193D70901B367F900138A040084
:105EC00063FEA700B3878700138AF4FF63E88700A7
:105ED00063F6A700138AE4FFB3878700B384A74063
:105EE00093850A0013850400EF201036130905007E
:105EF00093850A0013850400EF20903093990901DF
:105F000093040500930505001319090113850B007F
:105F100093D90901EF20102CB369390113860400CD
:105F200063FCA900B30934011386F4FF63E689001A
:105F300063F4A9001386E4FF13140A013364C40058
:105F4000130A00006F000013B707000113070001D8
:105F5000E36CF6EE130780016FF01FEF138A060063
:105F6000631A06009305000013051000EF20502966
:105F700013040500B7070100637EF4129307F00FC6
:105F800063F48700130A8000B35744013309F90012
:105F9000034709009306000233074701B386E64032
:105FA00063940612B3848440130A1000135B040147
:105FB00093050B0013850400EF2010291309050039
:105FC00093050B0013850400931B0401EF2050235D
:105FD00093DB0B01930405009305050013850B006B
:105FE000EF20501F1319090193D70901B367F90076
:105FF000938A040063FEA700B3878700938AF4FFA7
:1060000063E8870063F6A700938AE4FFB3878700FD
:10601000B384A74093050B0013850400EF20D02222
:106020001309050093050B0013850400EF20501D94
:1060300093990901930405009305050013190901BB
:1060400013850B0093D90901EF20D018B3693901EA
:106050001386040063FCA900B30934011386F4FF1E
:1060600063E6890063F4A9001386E4FF13940A0130
:106070003364C4001305040093050A008320C102A1
:106080000324810283244102032901028329C101DF
:10609000032A8101832A4101032B0101832BC100C3
:1060A000032C8100832C4100032D01001301010307
:1060B00067800000B7070001130A0001E366F4ECF3
:1060C000130A80016FF05FEC3314D40033DAE4007C
:1060D000B399DA0033D7EA00935A0401B394D40099
:1060E00093850A0013050A00336B9700EF20D01543
:1060F0001309050093850A0013050A00931B040188
:10610000EF20101093DB0B019304050093050500AD
:1061100013850B00EF20100C1319090113570B0105
:106120003367E900138A0400637EA7003307870002
:10613000138AF4FF636887006376A700138AE4FF7D
:1061400033078700B304A74093850A001385040032
:10615000EF20900F1309050093850A0013850400B2
:10616000EF20100A930405009305050013850B002A
:10617000EF20500613170B011357070113190901DC
:10618000B367E9001387040063FEA700B3878700A5
:106190001387F4FF63E8870063F6A7001387E4FF23
:1061A000B3878700131A0A01B384A740336AEA0051
:1061B0006FF0DFDF63ECD51EB707010063F4F60470
:1061C0001307F00FB335D7009395350033D7B600DA
:1061D00097A7010093878715B387E70003C70700D8
:1061E000130A00023307B700330AEA4063160A02B3
:1061F00013041000E3E096E833B6CA001344160017
:106200006FF05FE7B707000193050001E3E0F6FCDC
:10621000930580016FF09FFBB35CE600B3964601E7
:10622000B3ECDC0033D4E40093DB0C01B3974401FE
:1062300033D7EA0093850B0013050400336BF70096
:10624000B3194601EF2050001309050093850B0098
:1062500013050400139C0C01EF20807A135C0C01E1
:10626000930405009305050013050C00EF208076CC
:106270001319090113570B013367E9001384040054
:10628000637EA700330797011384F4FF63689701C7
:106290006376A7001384E4FF33079701B304A74094
:1062A00093850B0013850400EF20007A1309050085
:1062B00093850B0013850400EF2080749304050080
:1062C0009305050013050C00EF20C07093170B0118
:1062D0001319090193D70701B367F9001386040066
:1062E00063FEA700B38797011386F4FF63E8970165
:1062F00063F6A7001386E4FFB38797011314040124
:10630000B70B01003364C4001389FBFF337D240104
:1063100033F92901B384A7409305090013050D0043
:10632000EF20406B935C040193050900130B0500FB
:1063300013850C00EF20006A93D90901130C0500A6
:106340009385090013850C00EF20C0681309050030
:106350009385090013050D00EF20C0673305850103
:1063600093570B013385A7006374850133097901C5
:1063700093570501B387270163E6F402E392F4BC67
:10638000B70701009387F7FF3375F5001315050173
:10639000337BFB0033964A0133056501130A000085
:1063A000E37AA6CC1304F4FF6FF09FB9130A000040
:1063B000130400006FF01FCC130101FB23248104A0
:1063C00023229104232E3103232291032326110437
:1063D00023202105232C4103232A51032328610371
:1063E00023267103232481032320A103232EB1013B
:1063F000930C0500938905001304050093840500A0
:10640000639E062613090600138A060097AA010058
:10641000938ACAF163F4C514B70701006376F612D4
:106420009307F00F63F4C700130A8000B3574601C7
:10643000B38AFA0003C70A001305000233074701B5
:10644000330AE540630C0A00B395490133D7EC00E9
:1064500033194601B364B70033944C01935A0901D0
:1064600093850A0013850400EF20005E9309050060
:1064700093850A00131B090113850400EF2040587F
:10648000135B0B019305050013050B00EF208054EF
:106490009399090193570401B3E7F90063FAA70040
:1064A000B387270163E6270163F4A700B3872701B9
:1064B000B384A74093850A0013850400EF20C058D9
:1064C0009309050093850A0013850400EF204053CB
:1064D00013140401930505009399090113050B009A
:1064E00013540401EF20004F33E48900637AA400C1
:1064F00033042401636624016374A400330424017B
:106500003304A44033554401930500008320C104A3
:106510000324810483244104032901048329C10342
:10652000032A8103832A4103032B0103832BC10226
:10653000032C8102832C4102032D0102832DC10112
:106540001301010567800000B7070001130A00016D
:10655000E36EF6EC130A80016FF05FED631A06003C
:106560009305000013051000EF2080491309050072
:10657000B7070100637AF90E9307F00F63F4270160
:10658000130A8000B3574901B38AFA0003C70A000F
:1065900013050002B384294133074701330AE5405C
:1065A000E30E0AEA33194901B3DAE900B395490168
:1065B00033D7EC0093540901336BB70013850A00FD
:1065C00093850400EF20404893090500938504005B
:1065D000931B090113850A00EF20804293DB0B0116
:1065E0009305050013850B00EF20C03E9399090128
:1065F00093570B01B3E7F90033944C0163FAA700FA
:10660000B387270163E6270163F4A700B387270157
:10661000B38AA7409385040013850A00EF20C04287
:10662000930905009385040013850A00EF20403D7F
:106630009305050013850B00EF20C03993150B015E
:106640009399090193D50501B3E5B90063FAA50053
:10665000B385250163E6250163F4A500B385250113
:10666000B384A5406FF09FDFB7070001130A000154
:10667000E36AF9F0130A80016FF0DFF0E3E8D5E890
:10668000B707010063FCF604930BF00F33B5DB0092
:106690001315350033D7A60097A70100938707C9C4
:1066A000B387E70083CB070093050002B38BAB00F1
:1066B000338B7541631E0B0263E4360163EACC0041
:1066C0003384CC40B386D94033B58C00B384A64024
:1066D00013050400938504006FF05FE3B707000122
:1066E00013050001E3E8F6FA130580016FF09FFA45
:1066F000B3966601335D7601336DDD0033D47901E5
:10670000B395690133DC7C0193540D01336CBC00FB
:106710001305040093850400B31A6601EF20C0320C
:10672000130A0500938504001305040033996C01D6
:10673000931C0D01EF20C02C93DC0C011304050009
:106740009305050013850C00EF20C028131A0A01D9
:1067500013570C013367EA00130A0400637EA70095
:106760003307A701130AF4FF6368A7016376A70044
:10677000130AE4FF3307A701B309A7409385040078
:1067800013850900EF20402C9385040013040500B5
:1067900013850900EF20C02693050500930405002A
:1067A00013850C00EF20002393150C011314040132
:1067B00093D50501B365B4001387040063FEA500FB
:1067C000B385A5011387F4FF63E8A50163F6A5006F
:1067D0001387E4FFB385A501131A0A01B70C010062
:1067E000336AEA001384FCFFB3778A0033F48A002B
:1067F000B384A54013850700930504002326F10008
:10680000135A0A01EF20001D9309050093050400A7
:1068100013050A00EF20001C13DC0A01930D05008C
:1068200093050C0013050A00EF20C01A8327C1004E
:10683000130A050093050C0013850700EF2080194B
:106840003305B50113D709013307A7006374B701F6
:10685000330A9A01B70701009387F7FF93550701A1
:106860003377F70013170701B3F7F900B385450134
:10687000B307F70063E6B400639EB400637CF900DD
:1068800033865741B3B7C700B385A541B385F540FB
:1068900093070600B307F9403339F900B385B440D4
:1068A000B385254133947501B3D767013365F4008F
:1068B000B3D565016FF09FC5370810001308F8FFC6
:1068C000130101FEB378B80013D745019357D501E2
:1068D000232821011379F77F139738003378D800E4
:1068E000B3E7E70013D7460113183800232A9100B5
:1068F0001377F77F93D8F601232E11009356D60114
:10690000232C81002326310193D4F50133E30601C2
:1069100013153500131636003308E9406394143B11
:106920006354001F631207143367C3006314070C1A
:106930009306F07F13070800631CD830B3E6A70066
:1069400063980630930700001305000093968700B4
:1069500063DE0600130717009306F07F630CD774FD
:10696000B70680FF9386F6FFB3F7D7009396D7015B
:106970001355350033E5A6009306F07F93D7370013
:10698000631ED7003365F500930700006308050018
:10699000B70708001305000093040000B7061000B5
:1069A0009386F6FFB3F7D700B70610801377F77F0B
:1069B0009386F6FF13174701B3F7D700B3E7E70055
:1069C000370700801347F7FF8320C10103248101AB
:1069D0009395F401B3F7E70033E7B700832441014F
:1069E000032901018329C100930507001301010256
:1069F000678000009305F8FF639C05043306C5001B
:106A00003335A600B3876700B387A70013071000CC
:106A1000130506009396870063DC06221307170010
:106A20009306F07FE300D7F2B70680FF9386F6FF68
:106A3000B3F6D70093551500137515009397F6011B
:106A400033E5A50033E5A70093D716006F0040207B
:106A50001307F07F6314E80233E7A70063000762BF
:106A60001307F07F6F00C01E1307F07FE306E9FEF7
:106A7000370780003363E3009305080013078003A2
:106A8000634EB7061307F0016342B7041307000211
:106A90003307B740B356B6003318E3003316E600A9
:106AA0003368D8003336C0003368C800B355B3002C
:106AB0003308A800B385F500B337A800B387F50005
:106AC00013050800130709006FF0DFF41307000235
:106AD0003358B300930600006388E5009306000472
:106AE000B385B640B316B30033E6C6003336C000F4
:106AF0003368C800930500006FF09FFB3368C30044
:106B0000333800016FF01FFF630A080E631E090887
:106B1000B3E6A700639206029307F07F6318F700BD
:106B20003365C30093070000E30205E29307030007
:106B3000130506006F00C0119306F0FF631CD80018
:106B40003305C500B38767003336C500B387C70078
:106B50006FF05FEC9306F07F1348F8FFE302D7FC79
:106B60009306800363C606099306F00163CA06050F
:106B700093050002B3850541B3580501B396B700EC
:106B80003315B500B3E616013335A00033E5A60092
:106B900033D807013305C50033086800B337C50093
:106BA000B307F8006FF01FE79306F07FE30AD7F60C
:106BB000B706800033080041B3E7D7006FF05FFAF3
:106BC00093080002B3D6070193050000630818017B
:106BD0009305000433880541B395070133E5A5000B
:106BE0003335A00033E5A600130800006FF09FFACC
:106BF00033E5A7003335A0006FF01FFF130719001E
:106C00009375F77F9306100063C8B60833E7A700B3
:106C10006314090663080744B366C3001307000042
:106C2000638806023306C5003335A600B3876700C4
:106C3000B387A700939687001305060063DA060062
:106C4000370780FF1307F7FFB3F7E70013071000BC
:106C500093767500E38C06CE9376F500130640001C
:106C6000E386C6CE9306450033B5A600B387A700DA
:106C7000138506006FF09FCD630C073E3368C30099
:106C8000E30008DEB7074000130500001307F07F9C
:106C9000930400006FF09FCB9306F07FE304D7CA04
:106CA0003306C50033886700B337A6003308F80001
:106CB0001315F801135616003365C50093571800D5
:106CC0006FF01FF9635E000F6312070A3367C3009A
:106CD000E30007C69306F8FF639E06023306C5402D
:106CE0003335C500B3876740B387A740130710004B
:106CF0001305060093968700E3DC06F43704800052
:106D00001304F4FF33F48700930905001309070007
:106D10006F0000271307F07FE300E8D41307800318
:106D2000634AD7081307F001634ED7041307000224
:106D30003307D740B355D6003318E3003316E600C7
:106D40003368B8003336C0003368C800B356D30088
:106D500033080541B386D740B3370501B387F64002
:106D600013050800130709006FF0DFF81307F07F21
:106D7000E304E9CE370780003363E300930608009D
:106D80006FF0DFF9130700023358D300130400003B
:106D90006388E60013040004B306D4403314D30020
:106DA0003366C4003336C0003368C8009306000061
:106DB0006FF01FFA3368C300333800016FF01FFF14
:106DC000630A080E631E0908B3E6A7006390060273
:106DD0009307F07F6316F7003365C3006308052A45
:106DE00093070300130506006F00C00F9306F0FF22
:106DF000631ED8003305A640B307F3403336A60020
:106E0000B387C740938408006FF0DFEE9306F07FEE
:106E10001348F8FFE302D7FC9306800363C6060914
:106E20009306F00163CA060593050002B385054188
:106E3000335E0501B396B7003315B500B3E6C6015E
:106E40003335A00033E5A60033D807013305A6404B
:106E500033080341B337A600B307F8406FF09FFA39
:106E60009306F07FE30AD7F6B706800033080041A7
:106E7000B3E7D7006FF05FFA130E0002B3D6070135
:106E8000930500006308C801930500043388054199
:106E9000B395070133E5A5003335A00033E5A6001F
:106EA000130800006FF09FFA33E5A7003335A00008
:106EB0006FF01FFF130719001377F77F9306100079
:106EC00063CAE608B3E6A7003367C3006314090684
:106ED000639E06006302071C930703001305060068
:106EE00013070000938408006FF09FD66300070427
:106EF000B306C540B335D500338767403307B74085
:106F00009315870063DC05003305A640B307F34003
:106F10003336A600B387C7406FF09FFC33E5E60029
:106F2000630A050C9307070013850600130700008A
:106F30006FF01FD2639C06006308071693070300D7
:106F400013050600938408006FF09FB1E30A07B0B1
:106F50006FF05FD3B309C5403384674033383501E0
:106F6000330404411317840063520708B309A64091
:106F70003304F340B33736013304F44093840800FC
:106F8000630E040613050400EF105032130785FF4B
:106F90009307F00163CCE70693070002B387E7404D
:106FA0003314E400B3D7F90033E487003395E900E4
:106FB0006340270B33072741930717009306F0011F
:106FC00063CEF604130700023307F7403356F5008B
:106FD000B316E4003315E500B3E6C6003335A00070
:106FE00033E5A600B357F4006FF05FF433E5890092
:106FF000E31805F8930700006F00800A1385090065
:10700000EF10D02A130505026FF05FF8130485FD19
:1070100033948900130500006FF09FF9130717FEE2
:10702000130600023357E400930600006388C7008C
:1070300093060004B386F640B316D4003365D5003A
:107040003335A0003365A700930700006FF01FEEF3
:10705000B70780FF9387F7FF3307E940B377F40062
:107060006FF01FBF93070300130506006FF01FECBE
:1070700093070300130506006FF09F9E930700001F
:10708000130500001307F07F6FF05F8C930700007B
:10709000938408006FF09F8B930700001305000096
:1070A000130700006FF0DFBE13050000B7074000B4
:1070B0006FF0DFBD93070000130500006FF01F8B1A
:1070C000130101FB23248104232C41033704100006
:1070D00013DA450123202105232E3103232A5103EE
:1070E000232481031304F4FF232611042322910493
:1070F0002328610323267103232291032320A10364
:10710000232EB101137AFA7F13090500130C060030
:10711000938A06003374B40093D9F50163060A0A12
:107120009307F07F6304FA1013143400B70780004C
:107130003364F400135BD501336B8B00931435007B
:10714000130A1AC0930B000013D54A013709100027
:107150001309F9FF1375F57F3379590193050C0075
:1071600093DAFA01630205109307F07F6302F516C4
:107170003704800013193900336989001354DC0186
:107180003364240193153C00130515C093070000D8
:1071900013972B003367F7001307F7FF9306E00000
:1071A00033C95901330AAA4063E0E61697960100F5
:1071B00093864610131727003307D70003270700CD
:1071C0003307D70067000700336BA400630E0B067C
:1071D0006300040413050400EF10500D930755FFDE
:1071E0001307C001634CF702130BD001930485FF12
:1071F000330BFB4033149400335B6901336B8B001A
:10720000B3149900130AD0C0330AAA406FF09FF359
:10721000EF10D009130505026FF05FFC130485FD24
:10722000331B8900930400006FF0DFFD336BA40073
:1072300063040B0293040500130B0400130AF07F90
:10724000930B30006FF05FF093040000130A00000E
:10725000930B10006FF05FEF93040000130AF07FB0
:10726000930B20006FF05FEE33648901630E040618
:107270006300090413050900EF105003930755FF3D
:107280001307C001634EF7021304D001930585FF75
:107290003304F4403319B90033548C0033642401AF
:1072A000B315BC001307D0C03305A7406FF01FEE25
:1072B00013050C00EF10807F130505026FF01FFC13
:1072C000130485FD33148C00930500006FF09FFDBF
:1072D0003364890163020402130409001305F07F7B
:1072E000930730006FF0DFEA9305000013050000FC
:1072F000930710006FF0DFE9930500001305F07F9E
:10730000930720006FF0DFE86366640163128B4827
:1073100063E0B4489316FB0113D71400139CF401E7
:10732000135B1B00B3E4E6001314840093DC8501B7
:10733000B3EC8C0093DA0C0193970C0193D70701FF
:10734000139D850013050B0093850A002322F1008D
:10735000EF10006B93050500930B050013950C01CE
:1073600013550501EF1000671304050093850A000B
:1073700013050B00EF10406D1315050113D7040121
:107380003365A70093890B00637E85003305950163
:107390009389FBFF63689501637685009389EBFF12
:1073A000330595013304854093850A0013050400D5
:1073B000EF10006593050500930B050013950C0174
:1073C00013550501EF100061130B050093850A00AA
:1073D00013050400EF104067939D04011315050188
:1073E00093DD0D01B3EDAD0013870B0063FE6D015E
:1073F000B38D9D011387FBFF63E89D0163F66D016B
:107400001387EBFFB38D9D0193960901B70401002B
:10741000B3E6E600B38D6D41138BF4FF33F76601DD
:10742000337B6D011305070093050B0013D4060190
:107430002326D1002324E100EF10C0592322A1000C
:1074400093050B0013050400EF10C058935B0D016A
:107450009309050093850B0013050400EF10805776
:10746000032781001304050013850B009305070013
:10747000EF10405603264100330535018326C10035
:10748000135706013307A7006374370133049400D0
:10749000370501001305F5FF93540701B379A700E1
:1074A000939909013376A600B3848400B389C90097
:1074B00063E89D001384060063949D0463723C0599
:1074C000330CAC013337AC0133079701B38DED00BA
:1074D0001384F6FF63E6BC016394BC036362AC03F0
:1074E00063E69D00639EB401637C3C01330CAC01F8
:1074F0003337AC01330797011384E6FFB38DED00FA
:10750000B3093C41B3849D40B3373C01B384F4409C
:107510009305F0FF63889C1A93850A001385040085
:10752000EF10004E930505002324A10013950C01D4
:1075300013550501EF10004A2322A10093850A008C
:1075400013850400EF10405083268100032741007B
:107550001315050193D7090133E5A700938D0600A4
:10756000637EE50033059501938DF6FF6368950111
:107570006376E500938DE6FF33059501B304E5409E
:1075800093850A0013850400EF10804793050500DA
:107590002322A10013950C0113550501EF10804320
:1075A000130C050093850A0013850400EF10C049F1
:1075B00093990901032741001315050193D9090186
:1075C00033E5A90093070700637E85013305950124
:1075D0009307F7FF63689501637685019307E7FFDB
:1075E0003305950193940D01B3E4F40093970401DE
:1075F00093D7070193050B00B30985411385070055
:107600002322F10093DD0401EF10C03C93050B0031
:10761000930A050013850D00EF10C03B130C050005
:1076200093850D0013850B00EF10C03A83274100AE
:10763000130B050013850B0093850700EF108039AD
:107640003305850193D70A013385A7006376850149
:10765000B7070100330BFB00B70601009386F6FF66
:10766000935705013377D50013170701B3FADA00F2
:10767000B38767013307570163E8F9009385040076
:107680006390F9046300070433853C019385F4FF9C
:10769000636495036366F5006314F5026370ED029D
:1076A00093161D0033BDA601B30C9D019385E4FF25
:1076B00033059501138D06006314F5006304A701DB
:1076C00093E515001307FA3F6352E01293F7750034
:1076D0006380070293F7F50093064000638AD700A2
:1076E00093864500B3B5B6003304B4009385060015
:1076F0009317740063DA0700B70700FF9387F7FF5B
:107700003374F40013070A409307E07F63C2E71A5B
:107710009317D40193D53500B3E7B7001354340061
:10772000B70610009386F6FF3374D400B7061080B6
:107730001377F77F9386F6FF131747013374D4004E
:107740001319F9013364E400336724018320C10471
:107750000324810483244104032901048329C103F0
:10776000032A8103832A4103032B0103832BC102D4
:10777000032C8102832C4102032D0102832DC101C0
:1077800013850700930507001301010567800000BA
:10779000130AFAFF130C00006FF01FB913890900D8
:1077A00013040B009385040093870B00130720003C
:1077B0006380E710130730006382E70E13071000A1
:1077C000E392E7F013040000930700006F00400904
:1077D00013890A006FF09FFD37040800930500002D
:1077E00013090000930730006FF05FFC9306100050
:1077F000B386E64093078003E3C6D7FC9307F00106
:1078000063C4D706130AEA41B317440133D7D5003E
:10781000339A4501B3E7E700333A4001B3E7470144
:107820003354D40013F777006300070213F7F7000F
:1078300093064000630AD70013874700B337F70069
:107840003304F4009307070013178400634A070604
:107850001317D40193D73700B367F70013543400DC
:10786000130700006FF0DFEB930710FEB387E740CC
:1078700013070002B357F400130500006386E60007
:10788000130AEA4333154401336AB500333A400121
:10789000B3E74701130400006FF0DFF83704080076
:1078A000930700001307F07F130900006FF05FE7F4
:1078B00013040000930700001307F07F6FF05FE6EA
:1078C0001304000093070000130710006FF05FE53A
:1078D00013D74501B70710009387F7FF13D8460168
:1078E00093080500930E05001377F77F1305F07FCB
:1078F00033F3B700130F0600B3F7D70093D5F501A4
:107900001378F87F93D6F601631AA700336E13013C
:107910001305E0FF630C0E0867800000631AA800DF
:1079200033E6C7001305E0FF630A0608678000001E
:10793000631007083365130113351500631608003B
:1079400033E6C70063000606631A0500638ED500A0
:10795000130510006396050067800000E39E06FE95
:107960001305F0FF67800000E344E8FE635A070157
:107970001305F0FFE38205FE130510006780000089
:10798000E3E867FC631AF300E364DFFD130500001E
:10799000E3E0EEFF6FF05FFCE36CF3FC1305000027
:1079A00067800000E31C05FE6FF09FFAE30AE8F62B
:1079B00013050000E30608F86FF05FF9E31807F815
:1079C00033651301133515006FF01FF813D7450108
:1079D000B70710009387F7FF13D8460193080500F7
:1079E000930E05001377F77F1305F07F33F3B7008D
:1079F000130F0600B3F7D70093D5F5011378F87F7E
:107A000093D6F601631AA700336E13011305200005
:107A1000630C0E0867800000631AA80033E6C700F5
:107A200013052000630A060867800000631007083A
:107A300033651301133515006316080033E6C700DC
:107A400063000606631A0500638ED5001305100057
:107A50006396050067800000E39E06FE1305F0FFB5
:107A600067800000E344E8FE635A07011305F0FF56
:107A7000E38205FE1305100067800000E3E867FC61
:107A8000631AF300E364DFFD13050000E3E0EEFF9B
:107A90006FF05FFCE36CF3FC1305000067800000EF
:107AA000E31C05FE6FF09FFAE30AE8F613050000F9
:107AB000E30608F86FF05FF9E31807F83365130180
:107AC000133515006FF01FF8130101FA232C810400
:107AD000232631053704100093D94501232A910448
:107AE00023206105232E7103232C81031304F4FF4B
:107AF000232E110423282105232441052322510587
:107B0000232A91032328A1032326B10393F9F97FA4
:107B100093040500930B0600138C06003374B40025
:107B200013DBF5016388090A9307F07F6386F91078
:107B30003709800013143400336424011359D5012C
:107B400033698900131D3500938919C0930C000017
:107B500013554C01370A1000130AFAFF1375F57F0D
:107B6000337A8A0193840B00135CFC0163040510D3
:107B70009307F07F6304F51637048000131A3A0068
:107B8000336A8A0013D4DB013364440193943B00CD
:107B9000130515C09307000013972C003367F700F7
:107BA000B389A9001307F7FF9306E000B34B8B01DD
:107BB000938A190063E0E616978601009386467360
:107BC000131727003307D700032707003307D70011
:107BD000670007003369A400630E0906630004040C
:107BE00013050400EF00906C930755FF1307C001C5
:107BF000634CF7021309D001130D85FF3309F940D7
:107C00003314A40133D9240133698900339DA401BD
:107C10009309D0C0B389A9406FF05FF3EF001069FA
:107C2000130505026FF05FFC130985FD33992401EC
:107C3000130D00006FF0DFFD3369A4006304090237
:107C4000130D0500130904009309F07F930C300015
:107C50006FF01FF0130D000093090000930C10004B
:107C60006FF01FEF130D00009309F07F930C2000BD
:107C70006FF01FEE33647A01630E040663000A049A
:107C800013050A00EF009062930755FF1307C00128
:107C9000634EF7021304D001930485FF3304F440CC
:107CA000331A9A0033D48B0033644401B3949B009D
:107CB0009307D0C03385A7406FF0DFED13850B002D
:107CC000EF00D05E130505026FF01FFC130485FD65
:107CD00033948B00930400006FF09FFD33647A01AE
:107CE0006302040213040A001305F07F93073000B7
:107CF0006FF09FEA93040000130500009307100043
:107D00006FF09FE9930400001305F07F93072000B4
:107D10006FF09FE837070100130AF7FF135C0D01AE
:107D200093DD0401337D4D01B3F4440193050D004F
:107D3000138504002328E100EF00D049930C0500CF
:107D40009385040013050C00EF00D0482326A10002
:107D500093850D0013050C00EF00D047130B0500B1
:107D600093050D0013850D00EF00D0468326C1005A
:107D700093D70C013305D5003385A7006376D50072
:107D800003270101330BEB009356050133754501C1
:107D9000B3FC4C0113150501B3079501935C040175
:107DA0003374440193050D0013050400232AD10008
:107DB0002326F100EF0010422328A10093050400C0
:107DC00013050C00EF001041130A050093850C0009
:107DD00013050C00EF001040130C050093050D0077
:107DE00013850C00EF00103F032701013305450107
:107DF00083264101935707013385A7006376450128
:107E0000B7070100330CFC0037060100935705014A
:107E1000338C87019307F6FF337AF5003377F70049
:107E2000131A0A01135D0901330AEA003379F900D4
:107E30003387460193050900138504002328E100D8
:107E4000232EC100EF00103993850400232CA100DC
:107E500013050D00EF001038232AA10093050D0033
:107E600013850D00EF0010379304050093050900FA
:107E700013850D00EF001036832641010327810191
:107E80003305D500935707013385A7006376D500E6
:107E90000326C101B384C400B70601009387F6FF2F
:107EA000935D0501B3849D00B37DF5003377F70042
:107EB0009305090013050400939D0D01B38DED009A
:107EC000232CD100EF00103193050400232AA100D8
:107ED00013050D00EF00103093050D00130405008D
:107EE00013850C00EF00102F130D050093050900FA
:107EF00013850C00EF00102E032741013305850088
:107F0000935707013385A700637685008326810197
:107F1000330DDD0083270101B70601009386F6FFCC
:107F2000330BFB00B377D5003377D7009397070166
:107F3000B387E700333A4B01B387870133844701A6
:107F4000330BBB0133079400B33DBB01B306B7014C
:107F500033BC87013334440193570501333797000D
:107F600033648C00B3BDB6013304F400B36DB701C4
:107F70003304B4013304A40193D77601131494009D
:107F80003364F4008327C10093149B00135B7B01CF
:107F9000B3E4F400B334900093979600B3E4640123
:107FA000B3E4F4009317740063D2071293D714005C
:107FB00093F41400B3E497009317F401B3E4F400CE
:107FC000135414001387FA3F6356E01093F77400BC
:107FD0006380070293F7F40093064000638AD7009A
:107FE00093874400B3B4970033049400938407004C
:107FF0009317740063DA0700B70700FF9387F7FF52
:108000003374F40013870A409307E07F63C6E718D0
:1080100093DA34009314D401B3E4540113543400BC
:10802000B70710009387F7FF3374F4009377F77F57
:10803000370710801307F7FF939747013374E40065
:10804000939BFB013364F400B36774018320C10583
:1080500003248105138504000329010583244105B8
:108060008329C104032A8104832A4104032B0104C8
:10807000832BC103032C8103832C4103032D0103B4
:10808000832DC1029385070013010106678000005C
:10809000930B0B001304090093040D0093870C004D
:1080A00013072000638AE70E13073000638CE70C88
:1080B00013071000E398E7F0130400009304000096
:1080C0006F008008930B0C006FF09FFD938A0900EE
:1080D0006FF05FEF93061000B386E64093078003CE
:1080E000E3CCD7FC9307F00163C4D706938AEA4137
:1080F000B317540133D7D400B3945401B3E7E70066
:10810000B3349000B3E497003354D40093F7740071
:108110006380070293F7F40013074000638AE700C7
:1081200093874400B3B4970033049400938407000A
:108130009317840063CA07069317D40193D43400BD
:10814000B3E4970013543400130700006FF05FEDA1
:10815000930710FEB387E74013060002B357F400FD
:10816000130700006386C600938AEA43331754015D
:10817000B3649700B3349000B3E497001304000095
:108180006FF0DFF837040800930400001307F07F56
:10819000930B00006FF0DFE813040000930400006D
:1081A0001307F07F6FF0DFE7130400009304000073
:1081B000130710006FF0DFE6370810001308F8FF10
:1081C000130101FEB378B80013D745019357D501C9
:1081D0003378D800232821011379F77F13973800CB
:1081E000B3E7E70093D8F60113D746011318380018
:1081F0009356D601232A910033E30601232E110062
:10820000232C8100232631011377F77F9306F07F1B
:1082100093D4F50113153500131636006316D700F5
:10822000B366C3006394060093C818003308E9409E
:108230006394983A6354001F631207143367C300B2
:108240006314070C9306F07F13070800631CD830F3
:10825000B3E6A700639806309307000013050000FB
:108260009396870063DE0600130717009306F07FDE
:10827000630CD774B70680FF9386F6FFB3F7D70079
:108280009396D7011355350033E5A6009306F07F8A
:1082900093D73700631ED7003365F50093070000BE
:1082A00063080500B70708001305000093040000E9
:1082B000B70610009386F6FFB3F7D700B706108015
:1082C0001377F77F9386F6FF13174701B3F7D700AD
:1082D000B3E7E700370700801347F7FF8320C101AA
:1082E000032481019395F401B3F7E70033E7B70066
:1082F00083244101032901018329C100930507005B
:1083000013010102678000009305F8FF639C0504D8
:108310003306C5003335A600B3876700B387A700CF
:1083200013071000130506009396870063DC0622EE
:10833000130717009306F07FE300D7F2B70680FF1C
:108340009386F6FFB3F6D700935515001375150005
:108350009397F60133E5A50033E5A70093D7160000
:108360006F0040201307F07F6314E80233E7A70093
:10837000630007621307F07F6F00C01E1307F07FD2
:10838000E306E9FE370780003363E3009305080046
:1083900013078003634EB7061307F0016342B70467
:1083A000130700023307B740B356B6003318E30093
:1083B0003316E6003368D8003336C0003368C8008F
:1083C000B355B3003308A800B385F500B337A80050
:1083D000B387F50013050800130709006FF0DFF4F9
:1083E000130700023358B300930600006388E500CA
:1083F00093060004B385B640B316B30033E6C60057
:108400003336C0003368C800930500006FF09FFB4F
:108410003368C300333800016FF01FFF630A080E92
:10842000631E0908B3E6A700639206029307F07F74
:108430006318F7003365C30093070000E30205E209
:1084400093070300130506006F00C0119306F0FFA9
:10845000631CD8003305C500B38767003336C500F9
:10846000B387C7006FF05FEC9306F07F1348F8FF07
:10847000E302D7FC9306800363C606099306F00166
:1084800063CA060593050002B3850541B35805018B
:10849000B396B7003315B500B3E616013335A00027
:1084A00033E5A60033D807013305C500330868005B
:1084B000B337C500B307F8006FF01FE79306F07FEE
:1084C000E30AD7F6B706800033080041B3E7D700C8
:1084D0006FF05FFA93080002B3D60701930500001E
:1084E000630818019305000433880541B39507011B
:1084F00033E5A5003335A00033E5A60013080000DE
:108500006FF09FFA33E5A7003335A0006FF01FFF2F
:10851000130719009375F77F9306100063C8B60818
:1085200033E7A7006314090663080744B366C30072
:1085300013070000638806023306C5003335A60022
:10854000B3876700B387A7009396870013050600DB
:1085500063DA0600370780FF1307F7FFB3F7E7007A
:108560001307100093767500E38C06CE9376F50022
:1085700013064000E386C6CE9306450033B5A60039
:10858000B387A700138506006FF09FCD630C073EED
:108590003368C300E30008DEB7074000130500009E
:1085A0001307F07F930400006FF09FCB9306F07FDA
:1085B000E304D7CA3306C50033886700B337A60083
:1085C0003308F8001315F801135616003365C5007B
:1085D000935718006FF01FF9635E000F6312070ACC
:1085E0003367C300E30007C69306F8FF639E0602E5
:1085F0003306C5403335C500B3876740B387A7400E
:10860000130710001305060093968700E3DC06F4B9
:10861000370480001304F4FF33F487009309050046
:10862000130907006F0000271307F07FE300E8D469
:1086300013078003634AD7081307F001634ED7047A
:10864000130700023307D740B355D6003318E300B1
:108650003316E6003368B8003336C0003368C8000C
:10866000B356D30033080541B386D740B33705016D
:10867000B387F64013050800130709006FF0DFF811
:108680001307F07FE304E9CE370780003363E3008C
:10869000930608006FF0DFF9130700023358D30088
:1086A000130400006388E60013040004B306D440FA
:1086B0003314D3003366C4003336C0003368C800B7
:1086C000930600006FF01FFA3368C30033380001CF
:1086D0006FF01FFF630A080E631E0908B3E6A700C8
:1086E000639006029307F07F6316F7003365C300BB
:1086F0006308052A93070300130506006F00C00FE7
:108700009306F0FF631ED8003305A640B307F3407D
:108710003336A600B387C740938408006FF0DFEEBE
:108720009306F07F1348F8FFE302D7FC930680031B
:1087300063C606099306F00163CA060593050002A5
:10874000B3850541335E0501B396B7003315B50017
:10875000B3E6C6013335A00033E5A60033D80701E0
:108760003305A64033080341B337A600B307F840EA
:108770006FF09FFA9306F07FE30AD7F6B706800002
:1087800033080041B3E7D7006FF05FFA130E000221
:10879000B3D60701930500006308C80193050004E0
:1087A00033880541B395070133E5A5003335A000B3
:1087B00033E5A600130800006FF09FFA33E5A70029
:1087C0003335A0006FF01FFF130719001377F77FF1
:1087D0009306100063CAE608B3E6A7003367C30038
:1087E00063140906639E06006302071C93070300D7
:1087F0001305060013070000938408006FF09FD64E
:1088000063000704B306C540B335D500338767401E
:108810003307B7409315870063DC05003305A64096
:10882000B307F3403336A600B387C7406FF09FFC11
:1088300033E5E600630A050C93070700138506007D
:10884000130700006FF01FD2639C06006308071631
:108850009307030013050600938408006FF09FB18F
:10886000E30A07B06FF05FD3B309C54033846740B4
:108870003338350133040441131784006352070869
:10888000B309A6403304F340B33736013304F44050
:1088900093840800630E040613050400EF00002112
:1088A000130785FF9307F00163CCE70693070002E7
:1088B000B387E7403314E400B3D7F90033E487000B
:1088C0003395E9006340270B3307274193071700CF
:1088D0009306F00163CEF604130700023307F74056
:1088E0003356F500B316E4003315E500B3E6C600D1
:1088F0003335A00033E5A600B357F4006FF05FF402
:1089000033E58900E31805F8930700006F00800A3B
:1089100013850900EF008019130505026FF05FF859
:10892000130485FD33948900130500006FF09FF94F
:10893000130717FE130600023357E40093060000E6
:108940006388C70093060004B386F640B316D400CC
:108950003365D5003335A0003365A70093070000C9
:108960006FF01FEEB70780FF9387F7FF3307E940EB
:10897000B377F4006FF01FBF9307030013050600E1
:108980006FF01FEC93070300130506006FF09F9E26
:1089900093070000130500001307F07F6FF05F8C52
:1089A00093070000938408006FF09F8B93070000EB
:1089B00013050000130700006FF0DFBE1305000071
:1089C000B70740006FF0DFBD9307000013050000FC
:1089D0006FF01F8B130605001305000093F61500BA
:1089E000638406003305C50093D5150013161600E1
:1089F000E39605FE678000006340050663C6050632
:108A000013860500930505001305F0FF630C0602AD
:108A100093061000637AB6006358C0001316160060
:108A200093961600E36AB6FE1305000063E6C500E0
:108A3000B385C5403365D50093D61600135616008E
:108A4000E39606FE6780000093820000EFF05FFB74
:108A500013850500678002003305A04063D8050038
:108A6000B305B0406FF0DFF9B305B040938200006A
:108A7000EFF01FF93305A0406780020093820000E9
:108A800063CA0500634C0500EFF09FF713850500EE
:108A900067800200B305B040E35805FE3305A040EF
:108AA000EFF01FF63305B04067800200B707010002
:108AB000637AF5029307F00FB3B7A70093973700D7
:108AC000130700023307F740B357F500178501007D
:108AD0001305C585B307F50003C507003305A74097
:108AE000678000003707000193070001E36AE5FC97
:108AF000930780016FF0DFFC011122CC26CA2A8483
:108B0000AE844AC84EC652C456C206CEEF90CFAA13
:108B10001C4003290401B7090001B3E59700930A3B
:108B2000C4000CC08144FD19370A00021840638C50
:108B30002A03032609004A85B3654701B376360147
:108B400093175600758F0329490063C4070001E796
:108B5000F1BFE39DE6FC9317760063D30700D58C45
:108B6000EFA02F93E1B793C4F4FFF98C04C0EF900A
:108B7000AFC90840F2406244D2444249B249224A55
:108B8000924A056182804111014506C622C4EFC0A8
:108B9000FFBA17C7FFFF1307E72C81460546930569
:108BA0002003178501001305E58CEFA09FE219C98A
:108BB0002A84EF906FA12A86014781468545228548
:108BC000EFA0DFEDEF803FF8B240224401454101C4
:028BD0008280A1
:02000004800278
:100000005C45FEFF5A46FEFF6445FEFF5A46FEFF72
:100010005A46FEFF5A46FEFF5A46FEFF7C45FEFF4B
:100020005A46FEFF5A46FEFF9645FEFFA245FEFFDA
:100030005A46FEFFB445FEFFC045FEFFC045FEFF29
:10004000C045FEFFC045FEFFC045FEFFC045FEFFA8
:10005000C045FEFFC045FEFFC045FEFF5A46FEFFFD
:100060005A46FEFF5A46FEFF5A46FEFF5A46FEFF1C
:100070005A46FEFF5A46FEFF5A46FEFF5A46FEFF0C
:100080005A46FEFF5A46FEFF5A46FEFF5A46FEFFFC
:100090005A46FEFF5A46FEFF5A46FEFF5A46FEFFEC
:1000A0005A46FEFF5A46FEFF5A46FEFF5A46FEFFDC
:1000B0005A46FEFF5A46FEFF5A46FEFF5A46FEFFCC
:1000C0005A46FEFF5A46FEFF5A46FEFF5A46FEFFBC
:1000D0005A46FEFF5A46FEFF5A46FEFF5A46FEFFAC
:1000E0005A46FEFF5A46FEFF5A46FEFF5A46FEFF9C
:1000F0005A46FEFF5A46FEFF5A46FEFF5A46FEFF8C
:10010000F445FEFF0A46FEFF5A46FEFF5A46FEFF32
:100110005A46FEFF5A46FEFF5A46FEFF5A46FEFF6B
:100120005A46FEFF5046FEFF5A46FEFF5A46FEFF65
:100130000244FEFFBA44FEFF5A46FEFF5A46FEFF47
:10014000F044FEFF5A46FEFF4845FEFF5A46FEFFBA
:100150005A46FEFF7645FEFF6849FEFFBC49FEFF9A
:100160007049FEFFBC49FEFFBC49FEFFBC49FEFFD3
:10017000BC49FEFF6248FEFFBC49FEFFBC49FEFFD2
:100180007C48FEFF8848FEFFBC49FEFF9A48FEFF00
:10019000A648FEFFA648FEFFA648FEFFA648FEFFB3
:1001A000A648FEFFA648FEFFA648FEFFA648FEFFA3
:1001B000A648FEFFBC49FEFFBC49FEFFBC49FEFF4E
:1001C000BC49FEFFBC49FEFFBC49FEFFBC49FEFF27
:1001D000BC49FEFFBC49FEFFBC49FEFFBC49FEFF17
:1001E000BC49FEFFBC49FEFFBC49FEFFBC49FEFF07
:1001F000BC49FEFFBC49FEFFBC49FEFFBC49FEFFF7
:10020000BC49FEFFBC49FEFFBC49FEFFBC49FEFFE6
:10021000BC49FEFFBC49FEFFBC49FEFFBC49FEFFD6
:10022000BC49FEFFBC49FEFFBC49FEFFBC49FEFFC6
:10023000BC49FEFFBC49FEFFBC49FEFFBC49FEFFB6
:10024000BC49FEFFBC49FEFFBC49FEFFBC49FEFFA6
:10025000BC49FEFFBC49FEFFDA48FEFF0849FEFF2D
:10026000BC49FEFFBC49FEFFBC49FEFFBC49FEFF86
:10027000BC49FEFFBC49FEFFBC49FEFF5E49FEFFD4
:10028000BC49FEFFBC49FEFFC046FEFFBA47FEFF69
:10029000BC49FEFFBC49FEFF2C48FEFFBC49FEFFE7
:1002A0005248FEFFBC49FEFFBC49FEFFB649FEFFB7
:1002B0000076FEFF1475FEFF2075FEFF1475FEFF2D
:1002C000EC75FEFF1475FEFF2075FEFF0076FEFF45
:1002D0000076FEFFEC75FEFF2075FEFFEC74FEFF5E
:1002E000EC74FEFFEC74FEFF2875FEFFB47DFEFF8C
:1002F000B47DFEFFD87DFEFFA87DFEFFA87DFEFF3A
:10030000987EFEFFD87DFEFFA87DFEFF987EFEFF53
:10031000A87DFEFFD87DFEFFA47DFEFFA47DFEFF2D
:10032000A47DFEFF987EFEFF00010202030303038B
:100330000404040404040404050505050505050575
:100340000505050505050505060606060606060655
:10035000060606060606060606060606060606063D
:100360000606060606060606070707070707070725
:10037000070707070707070707070707070707070D
:1003800007070707070707070707070707070707FD
:1003900007070707070707070707070707070707ED
:1003A00007070707070707070808080808080808D5
:1003B00008080808080808080808080808080808BD
:1003C00008080808080808080808080808080808AD
:1003D000080808080808080808080808080808089D
:1003E000080808080808080808080808080808088D
:1003F000080808080808080808080808080808087D
:10040000080808080808080808080808080808086C
:10041000080808080808080808080808080808085C
:100420000808080808080808546D72510000000008
:10043000546D722053766300286E756C6C29000031
:100440004572726F7220696E20666C6F70732074D3
:1004500061736B73200D0A006D69616F750A00008E
:100460006D69616F75320A0068756E6772790A008E
:10047000436865636B54696D657200004D61746813
:10048000310000004D617468320000004D617468F5
:0C049000330000004D617468340000006F
:10049C001000000000000000017A5200017C0101F4
:1004AC001B0D02005000000018000000CC53FEFF92
:1004BC005805000000440E507489039406990B8172
:1004CC0001880292049305950796089709980A9A51
:1004DC000C9B0D036C010AC144C844C944D244D3DB
:1004EC0044D444D544D644D744D844D944DA44DB24
:1004FC00440E00440B0000004C0000006C00000097
:10050C00D058FEFFDC05000000440E3070890395C6
:10051C00078101880292049305940696089709981E
:10052C000A990B9A0C0370020AC144C844C944D2FC
:10053C0044D344D444D544D644D744D844D944DADB
:10054C00440E00440B00000050000000BC000000F2
:10055C005C5EFEFF0005000000440E5074880289AA
:10056C00039305990B8101920494069507960897BD
:10057C0009980A9A0C9B0D0320010AC144C844C96E
:10058C0044D244D344D444D544D644D744D844D993
:0C059C0044DA44DB440E00440B00000075
:100618006AE67F50274C41C15305A3923ADD5E40FC
:1006280082E2C7985B53A240B29DEFA7C6B18CC0C7
:10063800FCA9F1D24D62503FAE47E17A145678C01A
:10064800CDCCCCCC8CBCDF4039D6C56D340000C0D5
:10065800E5D022DBF93E2840E5D022DBF93E3840E0
:10066800AC1C5A643B2F4240E5D022DBF93E48409F
:100678001E85EB51B84E4E40AC1C5A643B2F52407D
:10068800C876BE9F1A375540E5D022DBF93E584060
:10069800022B8716D9465B40FCA9F1D24D6250BFA8
:1006A80000000000000016400000000000001A4092
:1006B8000000000000001E40000000000000214073
:1006C800000000000000234000000000000025405A
:1006D8000000000000002740000000000000294042
:1006E8000000000000002B400000000000002D402A
:0806F800FC8F0100040000006A
:040000058000004037
:00000001FF
